:100000000C94D4020C94F1020C94F1020C94F102C1
:100010000C94F1020C94F1020C94F1020C94F10294
:100020000C94F1020C94F1020C94BD250C94F10295
:100030000C94F1020C94F1020C94F1020C944D0317
:100040000C94F1020C94F3020C942F280C94F102FE
:100050000C94F1020C94FB240C941F250C94F102D7
:100060000C94F1020C94AF240C94F1020C94F10264
:100070000C94F1020C94F1020C94F1020C94F10234
:100080000C944F250C948D250C9473250C94F1023F
:100090000C94F1020829573F9F2D49CBA5310F76CB
:1000A000C73493F27E37D00D013AB60B613D2AAAD0
:1000B000AB3F0000003F800000004D503256322E12
:1000C0003236004003CF008A006700330019001069
:1000D000000C0008004003A0011501CF00670033A9
:1000E000002200190010001932204000000A0F14ED
:1000F000191E23282D0A0A4D6F6E6F7061636B20E5
:100100004C6974652056312E332020202843295411
:1001100052494E414D4943204D6F74696F6E2043E3
:100120006F6E74726F6C20476D6248202620436F9B
:10013000204B4720323030350A0A003F20666F726C
:100140002068656C700A0A0045452D526561642E71
:100150002E2E0A005253343835204164722028254F
:1001600075290A00537465702D2F446972206D6FD4
:1001700064650A004F7665726C6F6164210A004FF6
:1001800076657274656D7065726174757265210A49
:1001900000556E646572766F6C74616765210A0044
:1001A0006E3D20256C640A004F4B0A002563002D2C
:1001B000000A0025630025630044697361626C6571
:1001C0002045450A00456E61626C652045450A0080
:1001D00057726974652045450A00256420746F20B4
:1001E00025640A00256C6420746F20256C640A0065
:1001F000746F20256C640A004D6F746F72207374E5
:100200006F700A002B0A002D0A0054454D503A2009
:1002100025642020564F4C543A2025640A00464954
:10022000464F2D46696C6C3A2025750A00763D20B4
:1002300025640A00703D20256C640A00733D20256A
:10024000750A00256420000A000A00544D43343525
:10025000342052414D20746573742C2068697420D9
:100260007468652073706163652062617220746FC9
:100270002073746F702074686520746573742E0A1F
:10028000004572726F7220617420616464726573DC
:10029000732025642C20646174612025642C2073F4
:1002A000686F756C642062652025640A0052414DB8
:1002B00020746573742066696E69736865642C20A8
:1002C000256C7520746573747320706572666F7227
:1002D0006D65642E0A003F0A0A0056787878782007
:1002E0003D20564D415820282575202E2E2025755D
:1002F0002920282575290A004178787878203D2022
:10030000414D415820282575202E2E202575292065
:10031000282575290A004278787878203D20424FB8
:10032000572020282575202E2E20257529202825A8
:1003300075290A004678782020203D204672657194
:1003400075656E63792052616E676520303D6D6121
:10035000782E2031353D6D696E2E20282575290AAD
:1003600000492F4A2F4B787878203D2043757272D0
:10037000656E74202830202E2E20323535292066D7
:100380006F7220763D302C20763E302C20613E303E
:10039000202825752C2025752C202575290A0A0072
:1003A00053782E2E78203D2044697374616E636506
:1003B0002F5461726765742028256C64290A004DEA
:1003C00078202020203D2053746F70204D6F64658D
:1003D00020303D6E6F2C20313D686172642C2032DC
:1003E0003D736F667420282575290A004E2F4F2013
:1003F00020203D2046696E642053796E6320312FA2
:100400003020506F730A004720202020203D2041DB
:1004100075746F20526566205365617263680A00C7
:1004200050782E2E78203D2053657420506F730A2B
:1004300000442F522F54203D204472697665205687
:10044000656C6F63697479202F2052656C617469E3
:100450007665204D6F7665202F2054617267657434
:100460000A002B2F2D2020203D20446972656374E3
:10047000696F6E20282564290A00482F5820202003
:100480003D2048616C74202F2053746F7020616E82
:100490006420436C656172204572726F720A0A00B3
:1004A00043783D20436F6E74726F6C204D6F6465AE
:1004B00020303D7374642C20323D537465702F449A
:1004C000697220282575290A0059783D2050726FDD
:1004D000746F636F6C20303D7374642C20313D6DFC
:1004E000696E2C20322E2E393D5253343835202857
:1004F0002575290A005A783D205253343835204159
:10050000647220282575290A0055783D204D6963BD
:10051000726F737465702052657320303D32352CD4
:1005200020313D35302C20323D33322C20333D36C6
:100530003420282575290A0051783D204D697865B9
:100540006420446563617920303D6F66662C2031FC
:100550003D6F6E20282575290A0045203D20456EF7
:1005600061626C652F44697361626C65204545501A
:10057000524F4D0A0057203D205772697465207410
:100580006F20454550524F4D0A0A00642C662C7668
:100590002C702C73203D20446973706C6179207637
:1005A000616C7565730A000011241FBECFEFD0E1A6
:1005B000DEBFCDBF11E0A0E0B1E0E8EFFCE700E076
:1005C0000BBF02C007900D92AC33B107D9F714E00E
:1005D000ACE3B1E001C01D92AC3BB107E1F70C9474
:1005E0008E190C9400001F920F920FB60F921124D7
:1005F0002F933F934F938F939F9380910101817825
:10060000803811F0813039F480910001909101011E
:10061000880F991F07C08091000190910101880FF8
:10062000991F0196909301018093000140913C0134
:1006300080910001442331F099278F739070815489
:100640009F4F05C099278F719070815A9F4F90934B
:1006500099008093980020919800309199008091A2
:100660009400909195002817390738F480E880931A
:1006700092001092950010929400442311F080EEA5
:1006800001C080EF86BD9F918F914F913F912F9137
:100690000F900FBE0F901F9018951F920F920FB6DC
:1006A0000F9211242F933F938F939F9390913D012D
:1006B000992381F5659904C080915801813091F4A6
:1006C00080915B01882371F480910B01882321F0D4
:1006D000419A81E080935A015F9881E080935B01A9
:1006E00090935801809154018823A1F080914D018D
:1006F000882381F020915C01222361F480915001D4
:1007000090915101892B09F45F9881E080935C01FD
:1007100020934D01489B03C081E080935D0180914F
:100720000201882329F08091020181508093020107
:1007300080914E0190914F01892BA1F020914E01A3
:1007400030914F0180915001909151012817390744
:1007500048F480914E0190914F01019690934F0182
:1007600080934E0180914001883C39F48EB194E031
:1007700089278EB91092400105C0809140018F5F9A
:100780008093400180916901882329F0809169015B
:1007900081508093690180913E01882329F08091E6
:1007A0003E01815080933E0180913C01882319F0E5
:1007B00080EF98ED02C088E79CEE909385008093CF
:1007C00084009F918F913F912F910F900FBE0F90BA
:1007D0001F90189580913F01882351F0992781300F
:1007E0009105B9F00297C1F088B1837F88B9089567
:1007F0008FB186958695837099278330910534F45F
:10080000813091054CF4892B21F00895039761F311
:10081000089588B18C60EACF4298439A0895CF93A7
:10082000DF93EC01E0911601F0911701E05CFF4FBE
:1008300081E080830E947C24892B89F160E070E054
:1008400081E09FE00E9406220E947C24181619066F
:1008500034F4882799278C1B9D0BBC0101C0BE0175
:100860008AE092E00E94062260E070E08AE091E077
:100870000E940622E0911601F0911701E05CFF4F03
:1008800081E080830E947C24BC0181E893E00E9487
:10089000062260E070E08AE092E00E940622DF918A
:1008A000CF91089560E885E190E00E94DE2168EC38
:1008B00086E190E00E94DE216FEF87E190E00E94E8
:1008C000DE2160EA82E090E00E94DE216FE083E0BA
:1008D00090E00E94DE2168EE84E090E00E94DE213C
:1008E00063E085E090E00E94DE2164E686E090E02F
:1008F0000E94DE2160E087E090E00E94DE2160E05F
:1009000088E090E00E94DE2166E087E290E00E94AD
:10091000DE216AE081E190E00E94DE2160E082E178
:1009200090E00E94DE2160E08AE090E00E94DE21FB
:1009300064E689E090E00E94DE2161E08BE090E0D7
:100940000E94DE2160E08CE090E00E94DE2160E009
:100950008DE090E00E94DE2160E08EE090E00E9459
:10096000DE2160E489E190E00E94DE2160E08AE11E
:1009700090E00E94DE21939902C061E001C060E036
:1009800086E790E00E94DE2160E085E290E00E9430
:10099000DE2160E081E090E00E94DE2160E080E105
:1009A00090E00E94DE2160E084E190E00E94DE2180
:1009B00060E08BE190E00E94DE2160E08CE190E05D
:1009C0000E94DE2161E080E090E00E94DE2160E094
:1009D00082E390E00E94DE2160E083E390E00E94E9
:1009E000DE2160E084E390E00E94DE2160E085E3A8
:1009F00090E00E94DE2161E086E390E00E94DE212B
:100A000060E08DE190E00E94DE2160E08EE190E008
:100A10000E94DE2160E885E490E00E94DE2161E032
:100A200084E490E00E94DE2160E083E490E00E9494
:100A3000DE2160E082E490E00E94DE2160E081E45B
:100A400090E00E94DE2161E885E590E00E94DE21D1
:100A500062E084E590E00E94DE2160E083E590E0C2
:100A60000E94DE2160E082E590E00E94DE2160E0ED
:100A700081E590E00E94DE2160E080E690E00E9447
:100A8000DE2160E081E690E00E94DE2160E082E607
:100A900090E00E94DE2160E083E690E00E94DE218B
:100AA00060E084E690E00E94DE2160E085E690E070
:100AB0000E94DE2160E086E690E00E94DE2160E098
:100AC00087E690E00E94DE2160E088E690E00E94E8
:100AD000DE2160E089E690E00E94DE2160E08AE6A7
:100AE00090E00E94DE2160E08BE690E00E94DE2133
:100AF00060E08CE690E00E94DE2160E08DE690E010
:100B00000E94DE2160E08EE690E00E94DE2160E03F
:100B10008FE690E00E94DE2160E080E790E00E9496
:100B2000DE2162E088E290E00E94DE2162E082E75E
:100B300090E00E94DE2161E081E790E00E94DE21EA
:100B400064E083E790E00E94DE216FE084E790E0BC
:100B50000E94DE2160E085E790E00E94DE2162EEE7
:100B60008FE090E00E94DE210895CF92DF92EF9215
:100B7000FF920F931F93CF93C3B1C295CF70C095CF
:100B8000CF7082E190E00E94D0219927182F002792
:100B900081E190E00E94D0219927082B192B109316
:100BA00014010093130187E090E00E94D02199275F
:100BB000182F002786E090E00E94D0219927082B6B
:100BC000192B109312010093110183E090E00E9411
:100BD000D0219927182F002782E090E00E94D02191
:100BE0009927082B192B1093100100930F0185E012
:100BF00090E00E94D0219927182F002784E090E0F0
:100C00000E94D0219927082B192B10930E010093D5
:100C10000D0185E190E00E94D02180935D0486E182
:100C200090E00E94D02180934A0487E190E00E94E6
:100C3000D02180934804482F60914A0480915D043C
:100C40000E949E2387E290E00E94D0219927BC0158
:100C50008AE897E00E940622009116011091170180
:100C600084E390E00E94D0218375F801808B85E3B6
:100C700090E00E94D021E0911601F0911701858F3C
:100C800086E390E00E94D0218093570483E390E0B4
:100C90000E94D0219927182F002782E390E00E941C
:100CA000D0219927082B192B10934301009342015F
:100CB0008EE190E00E94D0219927182F00278DE126
:100CC00090E00E94D0219927082B192B1093450101
:100CD0000093440188E090E00E94D02110925F01CF
:100CE000109260011092610110926201282F332747
:100CF00021FF03C081E08093620122FF03C081E0F5
:100D00008093610123FF03C081E08093600124FF91
:100D100003C081E080935F0180916001882321F40A
:100D200081E08093620106C080916201882311F006
:100D300010925F0185E290E00E94D0219927182F40
:100D4000002781E090E00E94D021282F3327202B1C
:100D5000312B3093640120936301E0911601F091EF
:100D6000170190E080916001882319F0232B09F48A
:100D700091E097838AE090E00E94D0219927182F74
:100D8000002789E090E00E94D0219927082B192B99
:100D900010930A01009309018EE090E00E94D02197
:100DA0009927AA27BB27BA2FA92F982F8827809386
:100DB000050190930601A0930701B09308018DE00F
:100DC00090E00E94D021282F332744275527809177
:100DD000050190910601A0910701B0910801822BB5
:100DE000932BA42BB52BBA2FA92F982F882780934C
:100DF000050190930601A0930701B09308018CE0D0
:100E000090E00E94D0219927182F00278BE090E0D6
:100E10000E94D0219927082B192B9801442737FDD0
:100E20004095542F8091050190910601A0910701F2
:100E3000B0910801822B932BA42BB52B8093050135
:100E400090930601A0930701B093080189E190E017
:100E50000E94D021809304018AE190E00E94D02179
:100E600080934A0186E790E00E94D0218093490157
:100E700081E490E00E94D02182E490E00E94D021A1
:100E800083E490E00E94D0219927182F002784E462
:100E900090E00E94D0219927082B192B6801EE249D
:100EA000D7FCE094FE2CCC2331F4F1E0CF2ED12CF2
:100EB000E12CF12C10C080EF9FEFAFEFBFEFC82205
:100EC000D922EA22FB228C2F9927AA27BB27C82ADE
:100ED000D92AEA2AFB2AC0926B01D0926C01E092D7
:100EE0006D01F0926E0181E590E00E94D021C82E44
:100EF000DD24EE24FF24FE2CED2CDC2CCC2482E51A
:100F000090E00E94D0219927AA27BB27C82AD92A76
:100F1000EA2AFB2AFE2CED2CDC2CCC2483E590E085
:100F20000E94D0219927182F002784E590E00E9485
:100F3000D0219927082B192BC801AA2797FDA09526
:100F4000BA2FC82AD92AEA2AFB2ACC2329F452E04C
:100F5000C52ED12CE12CF12CC0926F01D0927001E2
:100F6000E0927101F092720181E790E00E94D0213D
:100F7000807F8C2B80935C04CC2319F481E08093D8
:100F80005C0482E790E00E94D02180934B0483E7C9
:100F900090E00E94D0218093490484E790E00E9471
:100FA000D02180935904809149040E94992680E0C1
:100FB00090E00E94D021982F917090930B01807146
:100FC0008093550180E190E00E94D02180934801F8
:100FD00084E190E00E94D021282F332720FF04C015
:100FE00081E08093540102C01092540121FF04C09B
:100FF00081E08093520105C022FF03C081E080930D
:10100000530180915201882321F480915301882358
:1010100091F08CE190E00E94D0219927182F0027B1
:101020008BE190E00E94D0219927082B192B109377
:1010300051010093500180E690E00E94D021E091A0
:101040001601F0911701E056FF4F808381E690E092
:101050000E94D021E0911601F0911701EF55FF4F4A
:10106000808382E690E00E94D021E0911601F09109
:101070001701EE55FF4F808383E690E00E94D02158
:10108000E0911601F0911701ED55FF4F808384E642
:1010900090E00E94D021E0911601F0911701EC55EB
:1010A000FF4F808385E690E00E94D021E0911601F9
:1010B000F0911701EB55FF4F808386E690E00E9488
:1010C000D021E0911601F0911701E855FF4F808380
:1010D00087E690E00E94D021E0911601F09117017F
:1010E000E755FF4F808388E690E00E94D021E09191
:1010F0001601F0911701E455FF4F808389E690E0D7
:101100000E94D021E0911601F0911701E355FF4FA5
:1011100080838AE690E00E94D021E0911601F09150
:101120001701E055FF4F80838BE690E00E94D021AD
:10113000E0911601F0911701EC54FF4F80838CE68B
:1011400090E00E94D021E0911601F0911701E8543F
:10115000FF4F80838DE690E00E94D021E091160140
:10116000F0911701E754FF4F80838EE690E00E94D4
:10117000D021E0911601F0911701E654FF4F8083D2
:101180008FE690E00E94D021E0911601F0911701C6
:10119000E454FF4F808380E790E00E94D021E091EB
:1011A0001601F0911701E354FF4F808385E790E02B
:1011B0000E94D02180933F01CF911F910F91FF900A
:1011C000EF90DF90CF900895EF92FF920F931F93CF
:1011D0008091460199278230910509F483C08330BC
:1011E00091051CF4019741F0DFC08330910591F126
:1011F000049709F483C0D8C00E941424DC01CB01F9
:10120000BC01CD010E94B61B7B018C0160E070E047
:101210008AE896E00E94062260E070E08AE892E0A8
:101220000E94062260E070E08AE893E00E940622B5
:10123000B801A7018DE80E94732260E070E082E8A7
:101240009FE00E940622809147018F5F80934701B3
:1012500083E051C0E0911601F0911701E05CFF4F6F
:1012600081E080830E94E023DC01CB0100916501D5
:1012700010916601209167013091680108171907E4
:101280002A073B07E4F480910D0190910E01442759
:101290005527481B590B809111019091120190958F
:1012A00081959F4FE0911301F0911401B0E8EB2E6E
:1012B000F12CBC01882799278E1B9F0B0FC0A0E83B
:1012C000EA2EF12C40910D0150910E016091110117
:1012D0007091120180911301909114010E94D72204
:1012E00082E009C084E00E94EF2185E00E94EF21A6
:1012F00083FD5AC084E08093460156C00E941424A6
:10130000DC01CB01BC01CD010E94B61B7B018C012D
:1013100080914401909145019C014427552780917B
:10132000650190916601A0916701B0916801821BEF
:10133000930BA40BB50BE816F9060A071B072CF153
:101340000E941424DC01CB01BC01CD010E94B61B1C
:101350007B018C0180914401909145019C014427BF
:1013600055278091650190916601A0916701B09128
:101370006801820F931FA41FB51F8E159F05A0073C
:10138000B1071CF01092460103C081E08093460132
:101390009091470180914801981730F010924601D2
:1013A00081E0809356015F981F910F91FF90EF901D
:1013B00008951F93CF93DF9380916001882351F0AC
:1013C00080916201882331F086E00E94EF21282F6E
:1013D00020710CC086E00E94EF21992724E09695A9
:1013E00087952A95E1F7282F2095217080915E013D
:1013F00099278530910509F4F0C08630910594F461
:101400008230910509F472C0833091051CF4019774
:10141000C9F050C28330910509F48CC0049709F4D7
:101420009AC048C28730910509F465C1873091059B
:101430000CF45CC18830910509F4A1C1099709F445
:1014400031C238C28091610120910D0130910E01AD
:101450004091110150911201882389F08827992722
:10146000821B930B909351048093500488279927F3
:10147000841B950B90935B0480935A0408C03093AF
:1014800051042093500450935B0440935A0482ED1E
:101490000E94EF218093580483ED0E94EF218093F6
:1014A0005604E0911601F0911701EE52FF4F1082A1
:1014B000E0911601F0911701ED52FF4F108284E088
:1014C0000E94EF2185E00E94EF2160E870E080E05B
:1014D00090E00E949622809160018823D1F186E0FD
:1014E0000E94EF2183FD35C082E0E2C184E00E94CA
:1014F000EF2185E00E94EF21E0911601F0911701A4
:10150000E05CFF4F81E08083809150049091510412
:10151000909581959F4F20915A0430915B0440E84B
:1015200050E0BC0188279927821B930B0E949E22C2
:1015300083E0BEC180916101882331F486E00E947E
:10154000EF2183FD06C0B6C186E00E94EF2182FF35
:10155000B1C184E0ADC184E00E94EF2185E00E942A
:10156000EF218091630190916401009751F460E84C
:1015700070E00E94962284E00E94EF2185E00E94A4
:10158000EF2140E850E06091500470915104809147
:101590005A0490915B040E949E22809162018823EC
:1015A00049F080916001882329F060E070E08FEFBE
:1015B0009FE004C060E070E08FED9FE00E94062293
:1015C00080916001882339F080916201882309F4B9
:1015D0006EC185E06DC189E06BC180916101882396
:1015E00031F486E00E94EF2183FD64C105C086E0EE
:1015F0000E94EF2182FD5EC10E94E023DC01CB014D
:1016000080934C0490934D04A0934E04B0934F04E8
:1016100010925E0180911101909112010E940F04BD
:1016200084E00E94EF2185E00E94EF21E091160105
:10163000F0911701E05CFF4F11E010830E94E0235E
:10164000DC01CB0120914C0430914D0440914E04BB
:1016500050914F04821B930BA40BB50BAC01BD0141
:101660008DE00E947322E0911601F0911701E05C79
:10167000FF4F108380E50E94EF21182F81E50E9423
:10168000EF21C82F82E50E94EF21E0911601F09131
:101690001701148BE0911601F0911701C58BE091B1
:1016A0001601F0911701868BE0911601F091170158
:1016B000EC52FF4F1082E0911601F0911701EB52AE
:1016C000FF4F84E08083E0911601F0911701EE5204
:1016D000FF4F809158048083E0911601F09117012B
:1016E000ED52FF4F809156048083E4C0222309F419
:1016F000E1C087E0DDC0222309F0DCC00E94E023C6
:10170000DC01CB0180934C0490934D04A0934E04D4
:10171000B0934F0480911101909112010E940F0427
:1017200084E00E94EF2185E00E94EF218091500427
:1017300090915104909581959F4F20915A0430913A
:101740005B0440E850E0BC0188279927821B930B7B
:101750000E949E2280916201882349F0809160015D
:10176000882329F060E070E08FEF9FE004C060E024
:1017700070E08FED9FE00E94062288E099C022234E
:1017800009F498C00E94E023DC01CB01809352044D
:1017900090935304A0935404B09355048091110185
:1017A000909112010E940F0484E00E94EF2185E0D5
:1017B0000E94EF21E0911601F0911701E05CFF4FCC
:1017C00011E010830E94E023FC01EB0120914C0406
:1017D00030914D0440914E0450914F048091520439
:1017E00090915304A0915404B0915504280F391FCF
:1017F0004A1F5B1F57FF04C02F5F3F4F4F4F5F4F84
:101800005595479537952795C21BD30BE40BF50BE0
:10181000AE01BF018DE00E947322E0911601F091AC
:101820001701E05CFF4F108380E50E94EF21182F25
:1018300081E50E94EF21C82F82E50E94EF21E0910F
:101840001601F0911701148BE0911601F091170128
:10185000C58BE0911601F0911701868BE09116017E
:10186000F0911701EC52FF4F1082E0911601F091B8
:101870001701EB52FF4F84E08083E0911601F09155
:101880001701EE52FF4F809158048083E0911601BA
:10189000F0911701ED52FF4F809156048083109212
:1018A0005E0108C086E00E94EF2184FD03C086E04F
:1018B00080935E01DF91CF911F910895FF920F9366
:1018C0001F93CF93DF9386E00E94EF2184FD3BC0FE
:1018D000E0911601F0911701E05CFF4F31E0F32E2B
:1018E000F0820E94E023DC01CB01BC0197FF03C022
:1018F000709561957F4F0091090110910A01600F69
:10190000711FEB01EE27FF2780916001882371F49E
:101910002091050130910601409107015091080185
:10192000BE01CF010E943F3EFC01EB01000F111FE1
:10193000C801AA27BB278C179D07AE07BF071CF459
:10194000F09259015F98DF91CF911F910F91FF9015
:101950000895AF92BF92CF92DF92EF92FF920F93D2
:101960001F93CF93009116011091170180E10E94FF
:10197000EF218062F801808BE0911601F091170150
:10198000E05CFF4FC1E0C0830E944824DC01CB0132
:10199000BC01CD010E94B61B5B016C010E94E023DB
:1019A0007B018C010E947C24892B31F180914201C2
:1019B000909143019C0144275527D801C701821B00
:1019C000930BA40BB50BA816B906CA06DB064CF0A0
:1019D0002E0D3F1D401F511F2A153B054C055D056F
:1019E0004CF480914C01882311F4C0934D01C093B5
:1019F0004C0102C010924C01CF911F910F91FF90AA
:101A0000EF90DF90CF90BF90AF9008950F931F930A
:101A1000CF93DF93CDB7DEB729970FB6F894DEBF2B
:101A20000FBECDBF90914B0499838A836B831C8238
:101A30001D821E821F8218861986082F11270635DF
:101A4000110509F47CC107351105ACF50531110507
:101A500009F4C0C006311105ACF40131110509F4D7
:101A60006BC0023111052CF40031110509F45CC082
:101A7000F9C20231110509F477C00431110509F4E6
:101A80007FC0F0C20135110509F4EEC00235110521
:101A90004CF40631110509F4BDC00731110509F4F4
:101AA000CBC0E0C20435110509F4F8C005351105B5
:101AB00009F418C1D7C20B36110509F4DAC10C3686
:101AC0001105CCF40935110509F488C10A35110551
:101AD0004CF40735110509F452C10835110509F414
:101AE00063C1C0C20336110509F48CC10A36110561
:101AF00009F49DC1B7C20037110509F433C201379B
:101B000011054CF40C36110509F4ECC10D36110524
:101B100009F405C2A7C20337110509F454C2013CF8
:101B2000110509F47FC29EC260FF03C080913F018E
:101B300025C085E790E020C060FF09C080915D046A
:101B40008C8380914A048D8380914804E6C185E1AD
:101B500090E00E94D0218C8386E190E00E94D02109
:101B60008D8387E190E0D7C160FF04C084E70E94C5
:101B7000EF2104C087E290E00E94D0218C8372C2E2
:101B800060FF16C0809111018C83809111019091AA
:101B90001201892F990F990B8D8380910F018E83EC
:101BA00080910F0190911001892F990F990B59C2C3
:101BB00086E090E00E94D0218C8387E090E00E9434
:101BC000D0218D8382E090E00E94D0218E8383E03B
:101BD00090E045C260FF0CC0809105018C8320918C
:101BE000050130910601409107015091080187C01D
:101BF0008BE090E00E94D0218C838CE090E00E94EA
:101C0000D0218D838DE090E00E94D0218E838EE0E4
:101C100090E025C260FF08C080910D018C83809107
:101C20000D0190910E01B4C084E090E00E94D0219B
:101C30008C8385E090E0F7C060FF09C080910401CB
:101C40008C8380914A018D8380914901BAC189E1D9
:101C500090E00E94D0218C838AE190E00E94D02104
:101C60008D8386E790E0ABC1862F99279C01217078
:101C7000307080FF06C080910B018C8380915501EC
:101C8000D4C0C9010E94D021282F332720FF02C0D1
:101C900081E08C8324FFE6C181E0C7C060FF0CC0F7
:101CA000809162018D83809161018E8380916001BA
:101CB0008F8380915F0114C188E090E00E94D02161
:101CC000282F332721FF02C081E08D8322FF02C02D
:101CD00081E08E8323FF02C081E08F8324FFC2C195
:101CE00081E0FEC060FF19C080916B018C83209160
:101CF0006B0130916C0140916D0150916E01BB27D9
:101D0000A52F942F832F8D83CA01AA27BB278E83EB
:101D1000852F9927AA27BB27A4C184E490E00E94BD
:101D2000D0218C8383E490E00E94D0218D8382E4D3
:101D300090E00E94D0218E8381E490E090C160FF0A
:101D40000CC080916F018C8320916F0130917001E4
:101D50004091710150917201D2CF84E590E00E94D0
:101D6000D0218C8383E590E00E94D0218D8382E591
:101D700090E00E94D0218E8381E590E070C160FFE9
:101D80000BC0809163018C83809163019091640109
:101D9000892F990F990B49C081E090E00E94D021D2
:101DA0008C8385E290E03FC060FF0BC080914801CA
:101DB0008C83809144018E838091440190914501F0
:101DC0001DC180E190E00E94D0218C838DE190E0E4
:101DD0000E94D0218E838EE190E041C160FF0AC055
:101DE000809109018C838091090190910A01892FCA
:101DF00099271BC089E090E00E94D0218C838AE063
:101E000090E011C060FF08C0809113018C83809125
:101E1000130190911401BCCF81E190E00E94D02188
:101E20008C8382E190E00E94D0218D831BC160FFF2
:101E30000EC080EA0E94EF218C8381EA0E94EF218C
:101E40008D8382EA0E94EF218E8383EA77C080E649
:101E500090E00E94D0218C8381E690E00E94D02106
:101E60008D8382E690E00E94D0218E8383E690E00D
:101E7000F6C060FF18C084EA0E94EF218C8385EAD7
:101E80000E94EF218D8388EA0E94EF218E8389EAE8
:101E90000E94EF218F838CEA0E94EF2188878DEAD0
:101EA0000E94EF211DC084E690E00E94D0218C8327
:101EB00085E690E00E94D0218D8386E690E00E9426
:101EC000D0218E8387E690E00E94D0218F8388E620
:101ED00090E00E94D021888789E690E00E94D0217E
:101EE0008987C0C060FF0CC084EB0E94EF218C8307
:101EF00080EB0E94EF218D8388EB0E94EF210DC0C3
:101F00008BE690E00E94D0218C838AE690E00E94CC
:101F1000D0218D83C8010E94D0218E83A3C060FF91
:101F200010C089EB0E94EF218C838AEB0E94EF2185
:101F30008D838CEB0E94EF218E838DEB0E94EF212D
:101F400090C0C8010E94D0218C838EE690E00E9450
:101F5000D0218D838FE690E00E94D0218E8380E790
:101F600090E07DC060FF15C080E10E94EF218C836E
:101F70008DE10E94EF218D83809142018E838091BB
:101F8000420190914301892F99278F8380915704B3
:101F900018C084E390E00E94D0218C8385E390E018
:101FA0000E94D0218D8382E390E00E94D0218E8315
:101FB00083E390E00E94D0218F8386E390E00E942B
:101FC000D02188874FC060FF1CC0809154018823B6
:101FD00011F081E08C8380915201882311F081E01F
:101FE0008D8380915301882311F082E08D8380914D
:101FF00050018E838091500190915101892F992732
:1020000030C084E190E00E94D021982F91709C8391
:1020100086958D838BE190E00E94D0218E838CE1A8
:1020200090E01DC060FF0AC0809149048C838091BC
:102030005C048D839E838091590413C083E790E0F4
:102040000E94D0218C8381E790E00E94D0218D8373
:1020500082E790E00E94D0218E8384E790E00E9486
:10206000D0218F8380916A01882329F4CE010196C3
:102070000E9428260BC0813029F4CE0101960E94CF
:102080008A2604C0CE0101960E94C91B29960FB66C
:10209000F894DEBF0FBECDBFDF91CF911F910F919E
:1020A0000895EF92FF920F931F93CF9380916A014F
:1020B000823041F09091600480915C04981711F097
:1020C0000C94881980910301882359F01092030120
:1020D0002091490140E060914A01809104010E94F1
:1020E000CF1E80916104082F11270335110509F4D3
:1020F000AFC4043511050CF079C00332110509F4A1
:1021000053C204321105CCF50531110509F487C11C
:1021100006311105BCF40131110509F4F3C0023197
:10212000110534F40031110509F4D2C00C9488195A
:102130000231110509F416C10431110509F42EC14B
:102140000C9488190032110509F417C201321105E7
:1021500054F40631110509F4B6C10731110509F42B
:10216000D9C10C9488190132110509F409C202324F
:10217000110509F408C20C9488190033110509F4FB
:102180000FC401331105BCF40732110509F4AEC3C5
:102190000832110534F40532110509F434C30C94E6
:1021A00088190A32110509F4E6C30B32110509F446
:1021B000F3C30C9488190035110509F4FAC30135ED
:1021C000110554F40334110509F4EDC30434110569
:1021D00009F4ECC30C9488190135110509F4FEC308
:1021E0000235110509F431C40C9488190D36110516
:1021F00009F4F6C60E361105A4F50835110509F4E3
:1022000089C50935110594F40535110509F48FC404
:10221000053511050CF41FC40635110509F4E5C494
:102220000735110509F441C50C9488190A361105C2
:1022300009F4ECC50B36110554F40935110509F400
:1022400097C50336110509F4BAC50C9488190B36E5
:10225000110509F423C60C36110509F487C60C9440
:1022600088190437110509F4BAC705371105BCF4FC
:102270000037110509F40DC70137110534F40F3685
:10228000110509F4F4C60C9488190137110509F4F5
:1022900052C70337110509F451C70C9488190C3C37
:1022A000110511F40C946D190D3C110554F4003C0A
:1022B000110509F4BDC7013C110509F4D2C70C94FE
:1022C00088190D3D110511F40C947D190C94881991
:1022D00060916204862F992781FD0EC0609163048E
:1022E00060933F0180FD04C085E790E00E94DE21FD
:1022F0000E94EA030C948819809161040E94060DE3
:102300000C94881960916204262F332721FD27C081
:102310006091630460935D048091640480934A0437
:10232000809165048093480420FD10C085E190E011
:102330000E94DE2160914A0486E190E00E94DE2145
:102340006091480487E190E00E94DE2140914804BA
:1023500060914A0480915D040E949E23D9C70E9427
:10236000060DD6C76091620461FD13C080916304BD
:102370009927BC018AE897E00E94062280916204B6
:1023800080FDC6C76091630487E290E00E94DE2171
:10239000BFC7809161040E94060DBAC760916204B4
:1023A000462F552741FD36C060916404862F99273A
:1023B000982F8827209163043327822B932B9093A7
:1023C000120180931101809166049927982F882724
:1023D000209165043327822B932B909310018093D7
:1023E0000F0140FD95C787E090E00E94DE216091DB
:1023F000630486E090E00E94DE216091660483E041
:1024000090E00E94DE216091650482E090E00E94ED
:10241000DE217EC7809161040E94060D79C760911C
:102420006204062F112701FD4BC080916604992795
:10243000AA27BB27BA2FA92F982F88272091650498
:10244000332744275527822B932BA42BB52B4427C6
:10245000582F692F7A2F809164049927982F882705
:10246000E09163042E2F3327822B932BAA2797FD0D
:10247000A095BA2F482B592B6A2B7B2B4093050133
:1024800050930601609307017093080100FD40C757
:102490006E2F8BE090E00E94DE21609164048CE05E
:1024A00090E00E94DE21609165048DE090E00E9442
:1024B000DE21609166048EE090E00E94DE2128C754
:1024C0000E94060D25C760916204462F552741FDE5
:1024D0001CC060916404862F9927982F882720912B
:1024E00063043327822B932B90930E0180930D016D
:1024F00040FD0EC785E090E00E94DE2160916304FC
:1025000084E090E00E94DE2103C7809161040E9474
:10251000060DFEC66091620461FD2AC0309163041D
:10252000309304019091640490934A018091670470
:1025300080934901282F40910301692F832F0E9426
:10254000CF1E8091620480FDE3C66091630489E13F
:1025500090E00E94DE21609164048AE190E00E9494
:10256000DE216091670486E790E00E94DE21D0C6FC
:10257000809161040E94060DCBC60E94381CC8C61B
:102580000E94481DC5C690915701992309F0C0C605
:1025900081E080935E019093460110924F0110926A
:1025A0004E0190934101B4C610915701112309F0D7
:1025B000AFC610924F0110924E0110934B01109331
:1025C0005E0110934601809166049927AA27BB27D4
:1025D000BA2FA92F982F88272091650433274427E5
:1025E0005527822B932BA42BB52BBA2FA92F982FCD
:1025F000882720916404332744275527822B932B67
:10260000A42BB52BBA2FA92F982F882720916304CC
:10261000332744275527822B932BA42BB52B80934C
:10262000650190936601A0936701B093680184E00F
:102630000E94EF2185E00E94EF21E0911601F091C8
:102640001701E05CFF4F81E080830E94D2239C0150
:102650002070387093FF02C0C12F06C0C0E860E848
:1026600070E0C9010E94962281E0809341010E949E
:10267000E023DC01CB012091650130916601281B2C
:10268000390B37FF03C0309521953F4F223031057C
:102690000CF47CC00E94E023DC01CB012091650199
:1026A00030916601281B390B37FF03C03095219507
:1026B0003F4F213131050CF069C00E94E0239B019E
:1026C000AC018091650190916601A0916701B09184
:1026D0006801EC2EFF2482179307A407B5078CF539
:1026E0000E94E023DC01CB010197A109B1092091EF
:1026F0000F013091100144275527421B530B2091A5
:1027000011013091120166277727621B730BE0914C
:102710001301F09114018C019D01882799278E1BCC
:102720009F0B0E94D7228091650190916601A09134
:102730006701B0916801AC01BD018EE00E94732277
:10274000E7C50E94E023DC01CB010196A11DB11D6C
:102750008C019D0140910F01509110016091110178
:102760007091120180911301909114010E94D7225F
:102770008091650190916601A0916701B091680117
:10278000AC01BD018EE00E947322C2C50E94E0230D
:10279000DC01CB0100916501109166012091670178
:1027A00030916801EC2EFF24081719072A073B0710
:1027B000DCF480910F019091100144275527481BAC
:1027C000590B8091110190911201909581959F4F25
:1027D000E0911301F0911401BC01882799278E1B09
:1027E0009F0B0E94D72294C540910F015091100178
:1027F0006091110170911201809113019091140167
:102800000E94D72285C580915701882309F080C591
:1028100010924F0110924E0180935E018093460109
:10282000809164049927182F0027809163049927C9
:10283000082B192B84E00E94EF2185E00E94EF21F4
:1028400080914101882361F060E870E080E090E0D1
:102850000E94962284E00E94EF2185E00E94EF21F1
:10286000E0911601F0911701E05CFF4F81E0808359
:102870000E947C2408171907F4F40E947C2460E06D
:1028800070E00E949622809111019091120140E81F
:1028900050E0B801909581959F4F0E949E2260E084
:1028A00070E08AE092E00E94062260E070E0C801D9
:1028B0000E9496222DC50E947C2460E070E00E9458
:1028C000962240E850E0B8018091110190911201E8
:1028D0000E949E2260E070E08AE092E00E94062260
:1028E00060E070E0C8010E94962212C580915E01EE
:1028F000882309F00DC510924F0110924E0180916E
:102900006604E82EFF2400271127102F0F2DFE2C20
:10291000EE24809165049927AA27BB27E82AF92A83
:102920000A2B1B2B102F0F2DFE2CEE2480916404FC
:102930009927AA27BB27E82AF92A0A2B1B2B102F35
:102940000F2DFE2CEE24809163049927AA27BB2724
:10295000E82AF92A0A2B1B2B80915704282F3327AA
:1029600044275527C801B7010E94613EC801B7013D
:102970000E940E23CDC410924F0110924E0110926E
:102980005E011092460180911101909112010E9406
:102990000F0410924101BCC481E080935801B8C477
:1029A0000E94AE1DB5C40E940B1CB2C40E94E81D5B
:1029B000AFC480916304813019F41092030103C005
:1029C00081E08093030120914901409103016091CE
:1029D0004A01809104010E94CF1E9AC46091620452
:1029E000262F3327A9014270507021FD29C0809104
:1029F000630480930B0160916404609355015093CC
:102A00005F0440935E04882331F081E090E090936E
:102A10005F0480935E04662349F080915E04909188
:102A20005F04409690935F0480935E04C9018170B7
:102A3000907020FD6DC460915E040E94DE2168C428
:102A4000809161040E94060D63C40E94A41C60C4AE
:102A50000E94DF1C5DC46091620461FD65C08091CD
:102A60006404809362018091650480936101909178
:102A70006604909360018091680480935F019923BC
:102A800029F481E080936201809364049091600155
:102A9000992341F080916201882321F010925F0117
:102AA00010926804E0911601F091170120E099233B
:102AB00039F08091630190916401892B09F421E040
:102AC00027838091620480FD23C480916404282FB1
:102AD0003327220F331F809165049927880F991F90
:102AE000880F991F282B809166049927A3E0880FEF
:102AF000991FAA95E1F7282B809168049927F4E0A3
:102B0000880F991FFA95E1F7282B80916304992784
:102B1000E5E0880F991FEA95E1F7282B622F88E0FE
:102B200090E00E94DE21F4C30E94060DF1C3609183
:102B30006204462F552741FD55C080916604E82E5A
:102B4000FF2400271127102F0F2DFE2CEE2480913B
:102B500065049927AA27BB27E82AF92A0A2B1B2BE9
:102B6000102F0F2DFE2CEE2480916304282F332785
:102B7000809164049927982F8827282B392BC90125
:102B8000AA2797FDA095BA2FE82AF92A0A2B1B2B12
:102B9000E0926B01F0926C0100936D0110936E0155
:102BA00040FDB6C36E2D84E490E00E94DE21BB2779
:102BB000A12F902F8F2D682F83E490E00E94DE21BB
:102BC000C801AA27BB27682F82E490E00E94DE217B
:102BD000812F9927AA27BB27682F81E490E00E94C4
:102BE000DE2196C30E94060D93C360916204462FB6
:102BF000552741FD55C080916604E82EFF2400272B
:102C00001127102F0F2DFE2CEE248091650499279B
:102C1000AA27BB27E82AF92A0A2B1B2B102F0F2DD6
:102C2000FE2CEE2480916304282F332780916404C6
:102C30009927982F8827282B392BC901AA2797FD78
:102C4000A095BA2FE82AF92A0A2B1B2BE0926F01D4
:102C5000F0927001009371011093720140FD58C30E
:102C60006E2D84E590E00E94DE21BB27A12F902FDE
:102C70008F2D682F83E590E00E94DE21C801AA27EE
:102C8000BB27682F82E590E00E94DE21812F9927E3
:102C9000AA27BB27682F81E590E00E94DE2138C378
:102CA000809161040E94060D33C36091620461FD4E
:102CB0002CC0809164049927382F222780916304C7
:102CC0009927282B392B3093640120936301E091DD
:102CD0001601F091170190E080916001882319F0AE
:102CE000232B09F491E097838091620480FD10C347
:102CF0006091630481E090E00E94DE2160916404B1
:102D000085E290E00E94DE2103C3809161040E946D
:102D1000060DFEC260916204462F552741FD25C075
:102D20006091630460934801809166049927982F0D
:102D30008827209165043327822B932B909345019C
:102D40008093440140FDE4C280E190E00E94DE21D6
:102D5000609165048DE190E00E94DE21609166043F
:102D60008EE190E00E94DE21D3C20E94060DD0C207
:102D700060916204462F552741FD1CC08091640478
:102D80009927982F882760916304262F3327822B59
:102D9000932B90930A018093090140FDB9C289E009
:102DA00090E00E94DE21609164048AE090E00E943D
:102DB000DE21AEC2809161040E94060DA9C260911D
:102DC0006204462F552741FD1CC080916404992759
:102DD000982F882760916304262F3327822B932B0B
:102DE000909314018093130140FD92C281E190E021
:102DF0000E94DE216091640482E190E00E94DE2165
:102E000087C2809161040E94060D82C260916204B3
:102E100061FD41C0E0911601F0911701E056FF4FAE
:102E2000809163048083E0911601F0911701EF55C2
:102E3000FF4F809164048083E0911601F0911701A7
:102E4000EE55FF4F809165048083E0911601F0916B
:102E50001701ED55FF4F80916604808380916204D5
:102E600080FD56C26091630480E690E00E94DE21FE
:102E70006091640481E690E00E94DE216091650427
:102E800082E690E00E94DE216091660483E690E095
:102E90000E94DE213DC20E94060D3AC2609162048A
:102EA00061FD5FC0E0911601F0911701EC55FF4FF5
:102EB000809163048083E0911601F0911701EB5536
:102EC000FF4F809164048083E0911601F091170117
:102ED000E855FF4F809165048083E0911601F091E1
:102EE0001701E755FF4F809166048083E09116013A
:102EF000F0911701E455FF4F809167048083E091C2
:102F00001601F0911701E355FF4F8091680480830B
:102F10008091620480FDFCC16091630484E690E0CE
:102F20000E94DE216091640485E690E00E94DE212B
:102F30006091650486E690E00E94DE21609166045F
:102F400087E690E00E94DE216091670488E690E0C9
:102F50000E94DE216091680489E690E00E94DE21F3
:102F6000D7C1809161040E94060DD2C160916204B4
:102F700061FD31C0E0911601F0911701EC54FF4F53
:102F8000809163048083E0911601F0911701E05570
:102F9000FF4F809164048083E0911601F091170146
:102FA000E854FF4F8091650480838091620480FD26
:102FB000AFC1609163048BE690E00E94DE216091D6
:102FC00064048AE690E00E94DE2160916504C801F5
:102FD0000E94DE219DC1809161040E94060D98C16E
:102FE0006091620461FD40C0E0911601F09117010B
:102FF000E754FF4F809163048083E0911601F091C4
:103000001701E654FF4F809164048083E09116011C
:10301000F0911701E454FF4F809165048083E091A3
:103020001601F0911701E354FF4F809166048083ED
:103030008091620480FD6CC160916304C8010E94AC
:10304000DE21609164048EE690E00E94DE216091B2
:1030500065048FE690E00E94DE216091660480E7BF
:1030600090E00E94DE2154C10E94060D51C1809162
:103070006304813039F462E070E08AE09EE00E94EF
:10308000062246C160E070E08AE09EE00E940622CF
:103090003FC16091620461FD4BC0E0911601F09167
:1030A0001701809163048375808BE0911601F09184
:1030B000170180916404858F809166049927982F69
:1030C0008827209165043327822B932B909343010B
:1030D000809342018091670480935704882319F4F8
:1030E00081E0809357048091620480FD11C180913A
:1030F00063048375682F84E390E00E94DE21609171
:10310000640485E390E00E94DE216091650482E31F
:1031100090E00E94DE216091660483E390E00E94CB
:10312000DE216091570486E390E00E94DE21F0C02A
:103130000E94060DEDC00E946C1CEAC05091620412
:1031400051FD47C060916304609354014091640451
:10315000413019F44093520108C01092520142309C
:1031600021F481E08093530102C010925301842F17
:103170008150823078F4809166049927982F8827AF
:10318000209165043327822B932B909351018093D8
:10319000500104C0109251011092500150FDB8C06E
:1031A0006170842F992783709070880F991F682B06
:1031B00084E190E00E94DE21609165048BE190E063
:1031C0000E94DE21609166048CE190E00E94DE2185
:1031D0009FC0652F809161040E94060D99C05F9A7F
:1031E0004198769A0E940E1DE0911601F091170108
:1031F000EC52FF4F8FEF8083E0911601F0911701A1
:10320000EB52FF4F808310925D0110925C0110928F
:10321000590110925B0110925801109257011092BF
:10322000560110924B01109275011092740170C0FA
:1032300060916304862F8150843020F488E290E00E
:103240000E94DE2180916B0190916C01A0916D0133
:10325000B0916E01AC01BD01809163040E94A92967
:1032600057C060916204862F992781FD31C060911B
:103270006304673008F04CC080FD16C083E790E01F
:103280000E94DE216091640481E790E00E94DE21CB
:103290006091650482E790E00E94DE2160916604FF
:1032A00084E790E00E94DE219091630490934904AA
:1032B0008091640480935C048091650480934B0446
:1032C0008091660480935904892F0E94992620C01A
:1032D000809161040E94060D1BC0F89488E190E083
:1032E00028E00FB6F894A895809360000FBE209355
:1032F0006000A4980C9400000BC08091630481339B
:1033000039F480916404813419F4A8950E94520420
:10331000CF911F910F91FF90EF900895CFEED0E1E4
:10332000DEBFCDBFDD240E94C52683E00E949F241E
:103330000E941F228FE090E00E94D021823E11F077
:103340000E9452040E94B505E0906B01F0906C0160
:1033500000916D0110916E0188E290E00E94D021F1
:10336000B801A7010E94A92981E08093030120915F
:103370004901482F60914A01809104010E94CF1EAB
:103380004198789480917A00806480937A0034998F
:1033900008C081E080933D0183E00E9499260E944D
:1033A000382B88E190E02FE00FB6F894A895809331
:1033B00060000FBE20936000A895369902C059980E
:1033C00001C0599A0E94EA0380916001882369F143
:1033D00080916301909164011816190634F580916B
:1033E0005E01882311F5E0911601F0911701E05C70
:1033F000FF4F81E080830E947C248C0197FF05C0F1
:1034000086E00E94EF2183FD08C0101611066CF4BF
:1034100086E00E94EF2182FF08C0809163019091B5
:1034200064010E940F041092410180915E01882383
:1034300019F00E94D9090AC080915F01882331F0F8
:1034400080915901882311F40E945E0C80915E01E5
:10345000882311F40E94A90C80911501882321F47E
:1034600080916A01882339F5CE0140960E94E925B2
:10347000882369F088E08D1550F0ED2DFF27E05A84
:10348000FB4F88898083D39484E68093690189E027
:10349000D81651F4DD24D0926901D0926A01D092FD
:1034A00015010E94511007C0DD2029F080916901AB
:1034B000882309F4D82E80911501882321F4809166
:1034C0006A01813041F5CE0140960E94372688235B
:1034D00069F088E08D1550F0ED2DFF27E05AFB4F85
:1034E00088898083D39484E68093690189E0D81623
:1034F00059F4DD24D092690181E080936A01D09271
:1035000015010E94511007C0DD2029F0809169014A
:10351000882309F4D82E80916A01823021F08091AD
:1035200015018823D1F0CE0101960E9449298823F4
:10353000A1F0A1E6B4E0FE01389697E081918D9369
:10354000915097FFFBCF8A818093470482E080935C
:103550006A01109215010E94511080915B0188232D
:1035600099F0E0905701EE2079F460E870E080E097
:1035700090E00E949622E0925E01E0924601E09285
:10358000410181E08093570180915D018823C1F062
:10359000809155018823A1F0E0905701EE2081F43D
:1035A00060E870E080E090E00E949622E0925E0188
:1035B000E0924601E092410181E0809357017698C4
:1035C00080917401882321F4809175018823A1F0F2
:1035D00060E870E080E090E00E94962210925E0128
:1035E000109246011092410181E080935701769834
:1035F000419A5F9880935A0180915C018823D1F1B0
:1036000090915301992321F480915201882391F1E3
:1036100080915201882339F080911101909112011B
:103620000E940F0408C0992331F060E870E080E048
:1036300090E00E94962210924601109241018091E2
:10364000500190915101892B91F020914B01809173
:103650004801281760F481E090E090934F01809337
:103660004E0110925C012F5F20934B0103C081E05B
:10367000809357012091500130915101211531055E
:1036800081F080914E0190914F018217930748F08D
:1036900010924F0110924E011092470181E08093E9
:1036A000460180914101882309F458C084E00E94BA
:1036B000EF2185E00E94EF2183FD50C0109241016F
:1036C00080914801882309F449C0109247010E9463
:1036D0001424DC01CB01BC01CD010E94B61B7B018F
:1036E0008C0180914401909145019C01442755270C
:1036F0008091650190916601A0916701B091680188
:10370000821B930BA40BB50BE816F9060A071B07DF
:1037100014F10E941424DC01CB01BC01CD010E94F4
:10372000B61B7B018C0180914401909145019C0165
:10373000442755278091650190916601A09167010A
:10374000B0916801820F931FA41FB51F8E159F05AE
:10375000A007B1071CF481E08093460180914601E7
:10376000882309F429CE0E94E40826CEDC01CB018F
:1037700020915704332744275527BC01CD010E94CF
:10378000203E97FD03C08F779070089580689F6FEB
:103790000895CF93DF93CDB7DEB72F970FB6F89488
:1037A000DEBF0FBECDBF28E029831B8220914704D6
:1037B0002A8320916F0130917001409171015091E5
:1037C00072012C833D834E835F83DE011896FC01DA
:1037D000319697E081918D93915097FFFBCFCE0169
:1037E00001960E9473292F960FB6F894DEBF0FBE84
:1037F000CDBFDF91CF91089520916A01222319F462
:103800000E9428260895213019F40E948A260895DE
:103810000E94C91B0895CF93DF93CDB7DEB72997D8
:103820000FB6F894DEBF0FBECDBF80914B048983E5
:1038300083E48A8382EE8B8380910C018C831D82CA
:1038400080916B048E8380916C048F8382E08887E3
:10385000198610920C01CE0101960E94FC1B29963C
:103860000FB6F894DEBF0FBECDBFDF91CF910895A4
:10387000CF93DF93CDB7DEB729970FB6F894DEBFAD
:103880000FBECDBFE0911601F0911701E05CFF4F34
:1038900081E0808380914B04898380E28A831B824C
:1038A00080E50E94EF218C8381E50E94EF218D83CA
:1038B00082E50E94EF218E831F8218861986CE0131
:1038C00001960E94FC1B29960FB6F894DEBF0FBE2E
:1038D000CDBFDF91CF910895CF93DF93CDB7DEB702
:1038E00029970FB6F894DEBF0FBECDBF0E941424F7
:1038F000DC01CB01BC01CD010E94B61B9B01AC01D8
:1039000080914B04898381E78A831B822C83BB27A8
:1039100057FDBA95A52F942F832F8D83CA01BB27FE
:1039200097FDB095AB2F8E831F8218861986CE0126
:1039300001960E94FC1B29960FB6F894DEBF0FBEBD
:10394000CDBFDF91CF910895CF93DF93CDB7DEB791
:1039500029970FB6F894DEBF0FBECDBF80914B0400
:10396000898382E58A831B8286E090E00E94D021D1
:103970008C8387E090E00E94D0218D8384E090E0EA
:103980000E94D0218E8385E090E00E94D0218F8319
:1039900082E090E00E94D021888783E090E00E943E
:1039A000D0218987CE0101960E94FC1B29960FB673
:1039B000F894DEBF0FBECDBFDF91CF910895CF93B6
:1039C000DF93CDB7DEB729970FB6F894DEBF0FBEF1
:1039D000CDBF80914B04898383E58A831B8285E177
:1039E00090E00E94D0218C8386E190E00E94D0215B
:1039F0008D8387E190E00E94D0218E831F821886FC
:103A00001986CE0101960E94FC1B29960FB6F894E8
:103A1000DEBF0FBECDBFDF91CF910895CF93DF936F
:103A2000CDB7DEB729970FB6F894DEBF0FBECDBF76
:103A300080914B04898384E78A831B8280915D0196
:103A40008C8380915C018D8380915B018E8380915A
:103A500059018F838091560188871986809175015D
:103A6000882311F081E0898780917401882319F0FF
:103A7000898582608987CE0101960E94FC1B299668
:103A80000FB6F894DEBF0FBECDBFDF91CF91089582
:103A9000EF92FF920F931F93CF93DF93CDB7DEB7D3
:103AA00029970FB6F894DEBF0FBECDBFE0905E0140
:103AB000EE2071F580914601882351F5E0911601C1
:103AC000F0911701E05CFF4F81E080838CE40E945D
:103AD000EF218DE40E94EF21F82E8EE40E94EF2169
:103AE000082F88E40E94EF2189E40E94EF21182F1B
:103AF0008AE40E94EF2190914B04998391E29A838A
:103B0000EB821C838D83FE820F83E886E98615C0D5
:103B100080914B04898381E28A831B821C821D82EF
:103B20001E821F82EE2011F48E2D01C08FEF888738
:103B30008091460181118FEF8987CE0101960E9405
:103B4000FC1B29960FB6F894DEBF0FBECDBFDF91E8
:103B5000CF911F910F91FF90EF900895CF93DF9336
:103B6000CDB7DEB729970FB6F894DEBF0FBECDBF35
:103B700086E00E94EF2190914B04998390E39A8311
:103B80001B82282F3327C90143E0969587954A95D4
:103B9000E1F781708C83C9019695879596958795F5
:103BA00081708D8324FF02C08B8101C081E08E83F0
:103BB0001F8218861986CE0101960E94FC1B299649
:103BC0000FB6F894DEBF0FBECDBFDF91CF91089541
:103BD000CF93DF93CDB7DEB729970FB6F894DEBF4A
:103BE0000FBECDBF80914B04898384E48A831B82FE
:103BF000809169048C8380916A048D8380916B0429
:103C00008E8380916C048F8318861986CE0101966D
:103C10000E94FC1B29960FB6F894DEBF0FBECDBFE5
:103C2000DF91CF910895EF92FF920F931F937B0145
:103C30008C012BED3FE049E45FE30E94BB3C88230D
:103C40002CF063EF74E085E39FE308C021E23BE7DB
:103C500046E65FE3C801B7010E94283D1F910F911E
:103C6000FF90EF900895DC01CB01BC01CD010E94D3
:103C7000703DDC01CB01BC01CD010895DC01CB011D
:103C800023E839EF42E25FE3BC01CD010E94283D09
:103C9000DC01CB01BC01CD0108956F927F928F9220
:103CA0009F92AF92BF92CF92DF92EF92FF920F93CB
:103CB0001F937B018C0159016A013B014C0120E0FB
:103CC00030E040E85FE30E94BB3C181654F40F2E2E
:103CD000F0E06F2EF0E07F2EF0E88F2EFFE39F2EB6
:103CE000F02D20E030E040E85FEBC801B7010E9412
:103CF000B83C882354F40F2EF0E06F2EF0E07F2EB6
:103D0000F0E88F2EFFEB9F2EF02D20E030E040E01A
:103D100050E0C801B7010E94BB3C18168CF4C601E4
:103D2000B5010E94331E7B018C01C601B5010E94C2
:103D3000131EDC01CB01A8019701BC01CD0110C00D
:103D4000C601B5010E94331E7B018C01C601B5017D
:103D50000E943E1EDC01CB019C01AD01C801B701F0
:103D60000E94083CDC01CB019C01AD01C401B30100
:103D70000E94283DDC01CB019C01AD01C801B701C7
:103D80000E94093C1F910F91FF90EF90DF90CF9020
:103D9000BF90AF909F908F907F906F9008952F92DB
:103DA0003F924F925F926F927F928F929F92AF92CB
:103DB000BF92CF92DF92EF92FF920F931F93CF9318
:103DC000DF93CDB7DEB760970FB6F894DEBF0FBEB6
:103DD000CDBF89836A834B832C83A0911601B09158
:103DE0001701813408F01EC288E8FD0180AFE09120
:103DF0001601F091170111AEE0911601F091170133
:103E000083E080ABE0911601F091170112AA222302
:103E100049F0939B07C0E0911601F09117018FE0E4
:103E200084AB05C0E0911601F091170114AAE0914E
:103E30001601F091170116AAF981AF2EBB24A7FC39
:103E4000B094CB2CDB2CC601B5010E94AE3C29817D
:103E500027FF06C020E030E040E853E40E94093C20
:103E600020E030E040E85FE30E94083CDC01CB0149
:103E700020E030E040E05FE3BC01CD010E94093C5E
:103E8000DC01CB012BED3FE049EC5FE3BC01CD0150
:103E90000E94283D7B018C01C601B5010E94AE3C09
:103EA000398137FF06C020E030E040E853E40E944B
:103EB000093C9B01AC01C801B7010E944B3C7B014E
:103EC0008C018A81992787FD9095A92FB92F8B871F
:103ED0009C87AD87BE87BC01CD010E94AE3CAA8104
:103EE000A7FF06C020E030E040E853E40E94093C10
:103EF00020E030E04EEF52E40E944B3CDC01CB016D
:103F0000A8019701BC01CD010E944D1EDC01CB012F
:103F10009C01AD0160E070E08FE793E40E944B3CB0
:103F2000DC01CB0120E030E040E05FE3BC01CD01EB
:103F30000E94093C6F83788789879A876624772453
:103F40007E826D82E981FF27F88BEF876E167F06F0
:103F50000CF092C0222433242101A0911601B091CB
:103F60001701A052BF4F8D812D813E812F5F3F4FA2
:103F70003E832D838C93A0911601B0911701398156
:103F8000323008F466C051EE852E912C8A0E9B1EAD
:103F9000C201B1010E94AE3CDC01CB012BED3FE040
:103FA00049EC5FE3BC01CD010E94283DDC01CB015F
:103FB00020E030E040E05FE3BC01CD010E94093C1D
:103FC0007B018C01C601B5010E94AE3CA981A7FF0F
:103FD00006C020E030E040E853E40E94093C9B0129
:103FE000AC01C801B7010E944B3C7B018C016B8581
:103FF0007C858D859E850E94AE3CBA81B7FF06C048
:1040000020E030E040E853E40E94093C20E030E04A
:104010004EEF52E40E944B3CDC01CB01A80197011A
:10402000BC01CD010E944D1EDC01CB012F813885E2
:1040300049855A85BC01CD010E94283DDC01CB0198
:10404000BC01CD010E94913CDC01CB01F4018083D5
:1040500004C0AF51BF4F84EB8C93A8950894611CAA
:10406000711C0894211C311C411C511C2F8538895E
:10407000621673060CF471CF3981432E5524320138
:1040800008946108710877200CF491C05301CC2486
:10409000B7FCC094DC2CA0911601B0911701A0527E
:1040A000BF4F8D81ED81FE813196FE83ED838C9330
:1040B000809016019090170121EE30E0820E931E41
:1040C000C601B5010E94AE3CDC01CB012BED3FE007
:1040D00049EC5FE3BC01CD010E94283DDC01CB012E
:1040E00020E030E040E05FE3BC01CD010E94093CEC
:1040F0007B018C013981832F992787FD9095A92F0A
:10410000B92FBC01CD010E94AE3CA981A7FF06C01A
:1041100020E030E040E853E40E94093C9B01AC0100
:10412000C801B7010E944B3C7B018C01EA818E2FB4
:10413000992787FD9095A92FB92FBC01CD010E9429
:10414000AE3CFA81F7FF06C020E030E040E853E4DF
:104150000E94093C20E030E04EEF52E40E944B3CCC
:10416000DC01CB01A8019701BC01CD010E944D1ECD
:10417000DC01CB012F81388549855A85BC01CD01F1
:104180000E94283DDC01CB01BC01CD010E94913C85
:10419000DC01CB01F4018083A895089461087108C3
:1041A0000894A108B108C108D10877FE74CFE09146
:1041B0001601F0911701EC51FF4F440C551C842D52
:1041C00081508083E0911601F0911701EB51FF4F70
:1041D0001082A0911601B0911701AA51BF4FF98129
:1041E000FC93A0911601B0911701A851BF4FF15057
:1041F000FC93E0911601F0911701E751FF4F1082F7
:10420000A0911601B09117012B81222311F088EAA9
:1042100001C088E8FD0180AFE0911601F09117011F
:1042200082E087C08CE8FD0180AFE0911601F0913B
:10423000170111AEFC81FF23C1F0939B16C0E091E2
:104240001601F09117018FEF84ABE0911601F09108
:10425000170186ABE0911601F091170180ABE09158
:104260001601F091170182AB14C0E0911601F09194
:10427000170114AAE0911601F091170116AAE09116
:104280001601F091170110AAE0911601F0911701A3
:1042900012AAE0911601F09117019FEF94A3E0910B
:1042A0001601F09117018FE185A3E0911601F091BD
:1042B000170196A3E0911601F09117018FE287A3F1
:1042C000E0911601F091170112AE2981822F9927F2
:1042D0008234910589F08334910524F48134910569
:1042E00029F016C08334910569F012C0E0911601DF
:1042F000F091170186E00BC0E0911601F0911701D3
:1043000087E005C0E0911601F091170188E086A7CB
:10431000A0911601B09117013B81332311F08CEA73
:1043200001C08CE8FD0180AFE0911601F09117010A
:1043300084E081AF939906C0FC81FF2311F040987F
:1043400001C0409A60960FB6F894DEBF0FBECDBF95
:10435000DF91CF911F910F91FF90EF90DF90CF9061
:10436000BF90AF909F908F907F906F905F904F9095
:104370003F902F9008958FB39927969587958095B4
:10438000909581709070089592BD81BD60BDFA9A3C
:10439000F99A089592BD81BDF89A80B5992708953C
:1043A000CF93DF93EC010E94BB218823E1F3CE0180
:1043B0000E94CA219927DF91CF9108951F93CF932F
:1043C000DF93EC01162F0E94BB218823E1F3612FBC
:1043D000CE010E94C421DF91CF911F910895982FA3
:1043E00080913C01882349F0E0911601F09117017A
:1043F000E90FF11D808180937301E0911601F09126
:104400001701E90FF11D808199270895E0911601A8
:10441000F09117018083892F9927E0911601F0917F
:1044200017018183E0911601F09117016283872FB4
:104430009927E0911601F09117018383089568E0B0
:1044400070E08AE097E00E94062261E070E088E078
:1044500090E00E94062261E070E088E091E00E9416
:1044600006226FEF7FE188E092E00E94062261E081
:1044700070E088E093E00E94062261E070E088E04E
:1044800094E00E94062261E070E088E095E00E94DE
:10449000062261E070E088E096E00E94062261E07A
:1044A00070E088E097E00E940622E0911601F0910A
:1044B0001701EC56FF4F1082E0911601F0911701A1
:1044C0008CEA80AFE0911601F091170185E081AF91
:1044D000E0911601F09117011782E0911601F09119
:1044E000170186A70895282FDB01CA01E091160164
:1044F000F09117012083E0911601F091170141839B
:10450000292F3A2F4B2F552747FD5A95E091160139
:10451000F09117012283CD01BB2797FDB095AB2FFA
:10452000E0911601F0911701838308959B01BC016E
:10453000C901826093600E94062208950F931F9321
:104540008B01BC01CA018A6092600E940622B801F8
:104550008AE091E00E94062260E070E081E09FE046
:104560000E9406221F910F910895EF92FF920F93E0
:104570001F93FC018B017A01C901BF018A6096601B
:104580000E940622B8018AE090E00E940622B7014C
:104590008AE091E00E94062260E070E080E09FE007
:1045A0000E9406221F910F91FF90EF9008956F9245
:1045B0007F928F929F92AF92BF92CF92DF92EF92B3
:1045C000FF920F931F93FC014B013A01C701BF01FA
:1045D0008A6096600E940622B4018AE090E00E9400
:1045E0000622B3018AE091E00E940622B901A801E7
:1045F0008EE00E94732260E070E083E09FE00E9402
:1046000006221F910F91FF90EF90DF90CF90BF9007
:10461000AF909F908F907F906F9008958F929F9210
:10462000AF92BF92CF92DF92EF92FF920F931F93C0
:104630005B016C0179018A0182ED0E94EF21982EC5
:1046400083ED0E94EF21882EE0911601F091170171
:10465000EE52FF4F1082E0911601F0911701ED52DA
:10466000FF4F108260E070E08AE896E00E94062228
:1046700060E070E08AE892E00E94062260E070E06C
:104680008AE893E00E940622B601A5018DE80E9407
:10469000732260E070E082E89FE00E94062260E002
:1046A00070E08FE89FE00E940622E0911601F091F1
:1046B0001701E48AE0911601F0911701BB2717FD5D
:1046C000BA95A12F902F8F2D858BE0911601F09137
:1046D0001701C801BB2797FDB095AB2F868BE091E2
:1046E0001601F0911701EC52FF4F1082E091160174
:1046F000F0911701EB52FF4F84E08083E0911601A7
:10470000F0911701EE52FF4F9082E0911601F09167
:104710001701ED52FF4F80821F910F91FF90EF9094
:10472000DF90CF90BF90AF909F908F900895992782
:10473000BC018AE097E00E9406220895FF920F9341
:104740001F93162FF42E9927BC0188E094E00E9455
:104750000622012F1127B80188E095E00E94062269
:10476000B80188E096E00E9406228F2D9927BC01AF
:1047700088E097E00E9406221F910F91FF90089514
:1047800060E070E082E093E00E940622089584E0F9
:104790000E94EF21882319F080E090E0089581E0E5
:1047A00090E008951F9384E00E94EF21182F85E088
:1047B0000E94EF21812F0E94EF2199271F910895D8
:1047C000DF92EF92FF920F931F9380E50E94EF21FB
:1047D000D82E82E50E94EF219927AA27BB278C01BA
:1047E000FF24EE2481E50E94EF219927AA27BB2709
:1047F0002227382F492F5A2F2E293F29402B512B62
:104800008D2D9927AA27BB27282B392B4A2B5B2BC9
:1048100047FF02C040685F6FCA01B9011F910F9145
:10482000FF90EF90DF900895DF92EF92FF920F9349
:104830001F9384E10E94EF21D82E86E10E94EF2190
:104840009927AA27BB278C01FF24EE2485E10E942B
:10485000EF219927AA27BB272227382F492F5A2F24
:104860002E293F29402B512B8D2D9927AA27BB2775
:10487000282B392B4A2B5B2B47FF02C040685F6F08
:10488000CA01B9011F910F91FF90EF90DF90089539
:10489000DF92EF92FF920F931F9388E10E94EF2126
:1048A000D82E8AE10E94EF219927AA27BB278C01E5
:1048B000FF24EE2489E10E94EF219927AA27BB2734
:1048C0002227382F492F5A2F2E293F29402B512B91
:1048D0008D2D9927AA27BB27282B392B4A2B5B2BF9
:1048E00047FF02C040685F6FCA01B9011F910F9175
:1048F000FF90EF90DF9008951F93CF93DF9388E4AC
:104900000E94EF21182F89E40E94EF21C82FDD2794
:104910008AE40E94EF2185FD806C9927982F8827D3
:10492000C82BD92BD7FD03C017FF04C002C0113814
:1049300008F02196CE01DF91CF911F9108958370E9
:104940008CBD8CB58C658CBD8DB581608DBD089599
:104950008EBD0DB407FEFDCF8EB5992708951F9229
:104960000F920FB60F9211242F938F939F938091E4
:104970007C008034D1F480917800909179009093FC
:104980006C0480936B0481E480937C00809102012D
:10499000882321F580916B0490916C04845A924095
:1049A000E8F081E08093740119C0809178009091C3
:1049B000790090936A048093690480E480937C007A
:1049C00080910201882351F48091690490916A04D6
:1049D0008455914018F481E08093750180917A00AC
:1049E000806480937A009F918F912F910F900FBEDA
:1049F0000F901F9018951F920F920FB60F921124CF
:104A00008F939F93EF93FF9390917C01E92FFF2762
:104A1000E258FE4F8091C60080839F5F90937C0197
:104A200080917C01823110F010927C01FF91EF9116
:104A30009F918F910F900FBE0F901F9018951F920E
:104A40000F920FB60F9211248F939F93EF93FF93C2
:104A500090917A0180917B01981799F080917A0169
:104A6000E82FFF27E057FE4F8F5F80937A01808108
:104A70008093C60080917A01823141F410927A01CC
:104A800005C08091C1008F7D8093C100FF91EF919F
:104A90009F918F910F900FBE0F901F9018951F92AE
:104AA0000F920FB60F9211248F939F93EF93FF9362
:104AB00090917801E92FFF27EE55FE4F8091CE00AF
:104AC00080839F5F9093780180917801823110F00C
:104AD00010927801FF91EF919F918F910F900FBEEF
:104AE0000F901F9018951F920F920FB60F921124DE
:104AF0008F939F939091760180917701981731F46D
:104B00005C988091C90080618093C9009F918F91CA
:104B10000F900FBE0F901F9018951F920F920FB617
:104B20000F9211248F939F93EF93FF9390917601AF
:104B300080917701981799F080917601E82FFF27EF
:104B4000EC54FE4F8F5F8093760180818093CE007E
:104B500080917601823141F41092760105C08091F6
:104B6000C9008F7D8093C900FF91EF919F918F9134
:104B70000F900FBE0F901F9018951F920F920FB6B7
:104B80000F9211248F938091C601882371F4809332
:104B9000B0008091C9008F7E8093C9005C9A80919B
:104BA000C90080628093C90005C08091C601815010
:104BB0008093C60180913C01882311F080EF01C0F1
:104BC00088EF8093B2008F910F900FBE0F901F90CF
:104BD0001895DC0190917D0180917C01981719F462
:104BE00080E090E0089580917D01E82FFF27E25852
:104BF000FE4F8F5F80937D0180818C9380917D013A
:104C0000823111F410927D0181E090E00895282F07
:104C100090917B019F5F923109F490E080917A013D
:104C20009817E1F380917B01E82FFF27E057FE4FB3
:104C300020838F5F80937B0180917B01823111F40F
:104C400010927B018091C10080628093C100089521
:104C50001F93CF93DF93EC0118E089910E94072600
:104C6000115017FFFACFDF91CF911F910895DC010A
:104C70009091790180917801981719F480E090E083
:104C8000089580917901E82FFF27EE55FE4F8F5F41
:104C90008093790180818C9380917901823111F424
:104CA0001092790181E090E00895282F909177018A
:104CB0009F5F923109F490E0809176019817E1F3BB
:104CC00080917701E82FFF27EC54FE4F20838F5F00
:104CD0008093770180917701823111F410927701EE
:104CE0005C9917C08091B000882399F48091590491
:104CF000882351F081508093C60180EF8093B200E9
:104D000087E08093B00008958091C900806280930D
:104D1000C90008951F93CF93DF93EC0118E08991A8
:104D20000E945526115017FFFACFDF91CF911F91A6
:104D3000089590913C01282F3327992389F0220F61
:104D4000331FF901EB52FF4F859194919093C50069
:104D50008093C400F901EB52FF4F8591949110C0EC
:104D6000220F331FF901ED53FF4F859194919093DA
:104D7000C5008093C400F901ED53FF4F85919491D4
:104D80009093CD008093CC000895CF93DF93CDB75F
:104D9000DEB722970FB6F894DEBF0FBECDBF27E077
:104DA00024B989EF85B99FE897B982E788B98AEB7A
:104DB0008AB982E88BB98EE48DB980EE8EB910BACB
:104DC0008CEF81BB85E183BB8BE184BB11B88FEF96
:104DD00082B99093740020937500A4980000A49A5F
:104DE00081E080933C0160E070E08FE89FE80E94E2
:104DF00006221A82198289819A81885B9B403CF441
:104E0000000089819A8101969A838983F4CFE09189
:104E10001601F0911701E05CFF4F81E0808384E48C
:104E20000E94EF2180936D0485E40E94EF2180931E
:104E30006E0486E40E94EF2180936F041092700448
:104E400080916D0490916E04A0916F04B0917004F4
:104E5000895C9F4AA040B04018F040E050E002C09A
:104E600041E050E040933C011092C50037E630939A
:104E7000C40022E02093C00088E98093C10096E03E
:104E80009093C2001092CD003093CC002093C800C4
:104E900088ED8093C9009093CA0081E080936F00F1
:104EA000442319F080EF98ED02C088E79CEE9093C0
:104EB0008500809384001092800082E080938100BE
:104EC0001092B00091E09093700084E084BD9093C4
:104ED0006E001092710090E49093900089E08093AE
:104EE000910090937C008EE880937A0022960FB612
:104EF000F894DEBF0FBECDBFDF91CF910895CF9361
:104F0000DF93FC01862F8295807F8093ED00809156
:104F1000EF0084FF03C081E0818301C01182809192
:104F2000EF008F7080838091F00082FF03C081E0EA
:104F3000828301C012828181882309F448C0809154
:104F4000F3009927AA27BB27C5E1880F991FAA1F3D
:104F5000BB1FCA95D1F783839483A583B6838091C1
:104F6000F200282F3327442755277DE0220F331FD7
:104F7000441F551F7A95D1F783819481A581B6810D
:104F8000822B932BA42BB52B83839483A583B68389
:104F90008091F100282F33274427552765E0220F01
:104FA000331F441F551F6A95D1F783819481A581D2
:104FB000B681822B932BA42BB52B83839483A5835B
:104FC000B6838091F0008695869586951DC0809168
:104FD000F3009927AA27BB2783839483A583B683ED
:104FE00083819481A581B68123E0880F991FAA1F30
:104FF000BB1F2A95D1F783839483A583B6838091C1
:10500000F200829586958770282F332744275527ED
:1050100083819481A581B681822B932BA42BB52B00
:1050200083839483A583B683DF0197E08091FA00A0
:10503000ED018F839150119697FFF8CF8091EE008C
:10504000809323041092EE008181882311F088E977
:1050500001C088E88093EF00DF91CF9108951F92FF
:105060000F920FB60F9211242F933F934F935F939C
:105070006F937F938F939F93AF93BF93EF93FF9320
:10508000CF93DF93CDB7DEB72197DEBFCDBF809141
:10509000DA00898389818F778093DA008091DC0040
:1050A00081FD1BC08091C7018F5F89838981843115
:1050B00009F4198299818091C801981771F0909133
:1050C000C7018FE0989FC001112461E089509D4F76
:1050D0000E947F2789818093C7018091DC0082FD37
:1050E0001BC08091C7018F5F89838981843109F456
:1050F000198299818091C801981771F09091C70128
:105100008FE0989FC001112462E089509D4F0E945A
:105110007F2789818093C7018091DC0080FDA2C038
:105120009091CA018091C901981731F48091DE00F5
:105130008E7F8093DE0096C08091CA019FE0899F98
:105140009001112425533E4F8F5F8093CA01109226
:10515000ED008091EE00809323041092EE00F9019F
:1051600097E087818093FA009150319697FFF9CFAD
:10517000F9018181882309F440C083819481A5814C
:10518000B681880F880F880F8093F0008381948107
:10519000A581B681689414F8B695A79597958795DB
:1051A0001694D1F78093F10083819481A581B68113
:1051B0006DE0B695A795979587956A95D1F78093F9
:1051C000F20083819481A581B681072E75E1B695A1
:1051D000A795979587957A95D1F7702D8093F300D1
:1051E0008281882329F08091F00084608093F00010
:1051F000F90180818F70806528C08093F0008093D2
:10520000F100F90183819481A581B6818295880F8F
:10521000807E8093F20083819481A581B681689419
:1052200012F8B695A795979587951694D1F7809320
:10523000F3008281882329F08091F00084608093BC
:10524000F000F90180818F7080648093EF0080917D
:10525000DE0081608093DE008091CA01843111F408
:105260001092CA012196F894DEBFCDBFDF91CF9195
:10527000FF91EF91BF91AF919F918F917F916F912E
:105280005F914F913F912F910F900FBE0F901F9004
:105290001895AC019091C8018091C701981719F435
:1052A00080E090E008952091C801822F9927FC01A9
:1052B000A4E0EE0FFF1FAA95E1F7E81BF90B2F5FA3
:1052C0002093C801DA01E950FD4F9FE001900D9253
:1052D0009150E1F78091C801843111F49093C80195
:1052E00081E090E00895AC012091C9012F5F243145
:1052F00009F420E08091CA01281741F18091C90189
:105300009927FC01B4E0EE0FFF1FBA95E1F7E81B07
:10531000F90BE553FE4FDA019FE00D900192915099
:10532000E1F72093C9018091DE0080FD0CC09093CD
:10533000ED008091EE0080648093EE008091DE00AD
:1053400081608093DE0081E090E0089580E090E04D
:105350000895982F1092DB0081E08093D80080910F
:10536000D80080FDFCCF1092CA018091CA018093C1
:10537000C9018091C9018093C8018091C8018093BF
:10538000C70120913C01892F99272223C9F082303F
:10539000910571F0833091051CF4019739F02DC00F
:1053A00083309105E1F00497E1F027C08EE001C061
:1053B00086E08093E20084E08093E3008EE31BC0EC
:1053C0008230910561F0833091051CF4019781F3DF
:1053D00014C08330910529F0049739F00EC082E0A3
:1053E000E8CF82E08093E20002C02093E20084E0F4
:1053F0008093E30082E18093E4008091E400816087
:105400008093E40020E09EE02093ED008091EE0088
:10541000809323041092EE001092EF009150205FD1
:1054200097FFF2CF1092ED008091EE00809323045D
:105430001092EE0080E18093ED008091EE00809369
:1054400023041092EE00DB01CA0123E0B695A79574
:10545000979587952A95D1F78093F300842F8295AD
:10546000880F807E8093F2001092F1001092F0007D
:105470002FEF2093F7002093F6002093F500209360
:10548000F40088E88093EF0080E28093ED00809143
:10549000EE00809323041092EE00DB01CA01F5E1D7
:1054A000B695A79597958795FA95D1F78093F300D0
:1054B000DB01CA01EDE0B695A79597958795EA952A
:1054C000D1F78093F200DB01CA0135E0B695A795CC
:1054D000979587953A95D1F78093F100842F880F9F
:1054E000880F880F8093F0002093F7002093F60038
:1054F0002093F5002093F40088E98093EF0086E084
:105500008093DE0080EB8093DB0082E08093D80004
:105510000895EF92FF920F931F937B018C0160E03F
:1055200070E082E89FE00E940622B801A7018DE8A2
:105530000E9473221F910F91FF90EF900895E091C8
:105540001601F091170180913904817087830895C5
:105550000F931F93CF938B01C22FBC01CA018A60A6
:1055600092600E940622B8018AE091E00E94062221
:1055700060E070E081E09FE00E940622CC2329F4E5
:1055800060E070E082E092E01AC0E0911601F091D4
:105590001701EC52FF4F80E88083E0911601F091F3
:1055A0001701EB52FF4F1082C13029F460E070E028
:1055B0008FEF90E004C060E070E08FED90E00E941B
:1055C0000622CF911F910F910895CF930E94D2236D
:1055D000C0E094FDC1E086E00E94EF2183FF0BC094
:1055E000E0911601F0911701E05CFF4F10820E94DC
:1055F0007C2497FDC1E086E00E94EF2182FF0DC070
:10560000E0911601F0911701E05CFF4F10820E94BB
:105610007C24181619060CF4C1E08C2F9927CF9121
:105620000895769A5F9A41981092460410927501F7
:105630001092740110925D010895CF93C82F80914C
:105640006A01882349F4CA3019F48DE00E940726C4
:105650008C2F0E94072608C0CA3019F48DE00E94E2
:1056600055268C2F0E94552680E090E0CF9108951A
:105670007F928F929F92AF92BF92CF92DF92EF92E2
:10568000FF920F931F93CF93DF93CDB7DEB7219790
:105690000FB6F894DEBF0FBECDBF772470926A01BB
:1056A00060E070E08DE19BE20E94623785EF90E060
:1056B0009F938F930E94BE370F900F908BE391E0E2
:1056C0009F938F930E94BE3780E091E00E94D0218B
:1056D0008093B1040F900F90863009F08DC088E45C
:1056E00091E09F938F930E94BE3781E091E00E94EA
:1056F000D0218093260182E091E00E94D021809306
:10570000270183E091E00E94D0218093240184E06E
:1057100091E00E94D0218093250185E091E00E94D4
:10572000D0218093220186E091E00E94D0218093D5
:10573000230187E091E00E94D0218093200188E03E
:1057400091E00E94D02180931F0189E091E00E94A6
:10575000D02180931E018AE091E00E94D0218093A5
:105760001D018BE091E00E94D021809321018CE00B
:1057700091E00E94D021809319018DE091E00E9478
:10578000D02180931A018EE091E00E94D021809375
:105790001B018FE091E00E94D02180931C0180E1E9
:1057A00091E00E94D0218093390481E191E00E9430
:1057B000D021809338040F900F90E82FFF27E551F8
:1057C000FF4F84918093590482E191E00E94D0219F
:1057D0008093370483E191E00E94D02180931801E7
:1057E00084E191E00E94D02180933A0485E191E028
:1057F0000E94D0218093360480913804823078F062
:105800008091180199279F938F9384E591E09F934E
:105810008F930E94BE370F900F900F900F90809142
:105820003A04823041F484E691E09F938F930E9482
:10583000BE370F900F9080913804823018F081E0CD
:1058400080936A010E941F22809120010E94972369
:105850000E949F2A40911D0160911E0180911F01AD
:105860000E949E2380913704E82FFF27E951FF4FC4
:105870009491472D80913A04823009F441E02091BF
:105880003604672D892F0E94CF1E80913A04E09143
:105890001601F0911701823029F4EC56FF4F84E095
:1058A000808303C0EC56FF4F70828EE380933F04E9
:1058B00088B1837F88B988E190E02FE00FB6F89433
:1058C000A895809360000FBE20936000A89536993C
:1058D00002C0599801C0599A80915D01882391F0C6
:1058E00010925D0176985F9880913804882351F476
:1058F000772041F484E791E09F938F930E94BE3715
:105900000F900F9080917401882321F4809175018C
:105910008823A1F110914604112381F560E870E01D
:1059200080E090E00E94962281E0809346041093EC
:1059300045041093320476985F98419A80935A01F7
:10594000809138048823D1F47720C1F480917401C8
:10595000882341F08FE791E09F938F930E94BE3799
:105960000F900F9080917501882341F081E991E0BB
:105970009F938F930E94BE370F900F900E94E52A4D
:1059800080934404882341F080913904823021F4CB
:1059900081E08093430404C01092430410924204B7
:1059A00080914304882309F463C0109142041123B9
:1059B00009F05EC0809342048091240190912501FA
:1059C00090932F0480932E0410923104109230048F
:1059D00060E070E082E89FE00E940622E0911601FC
:1059E000F0911701E05CFF4F10830E947C2490939C
:1059F0002D0480932C04809138048823D9F480915D
:105A00003004909131049F938F9380912C04909156
:105A10002D049F938F9388E291E09F938F930E9430
:105A2000A9374DB75EB74A5F5F4F0FB6F8945EBFB8
:105A30000FBE4DBF609130047091310480912C04F1
:105A400090912D04681779075CF480912E04909151
:105A50002F04909581959F4F90932F0480932E044F
:105A600040E850E080912E0490912F040E949E22E5
:105A700080914504813031F584ED0E94EF2187FF4C
:105A800021C0109245040E94E023DC01CB018093E9
:105A9000240490932504A0932604B0932704BF9375
:105AA000AF939F938F9380EA91E09F938F930E948F
:105AB000BE376DB77EB76A5F7F4F0FB6F8947EBF73
:105AC0000FBE6DBF80913204882309F468C0992706
:105AD00082309105D9F0833091051CF4019739F09B
:105AE0005EC08330910509F1049751F158C080914F
:105AF000210181958093210186E00E94EF2184FDA0
:105B000003C08EE480933F0482E017C08091450477
:105B1000882309F044C0809121018195809321015F
:105B20008FE480933F0483E008C08091450488237C
:105B3000B1F588E480933F0484E0809332042FC061
:105B400084E00E94EF21823050F50E94E023DC01C6
:105B5000CB012091240430912504409126045091DA
:105B60002704821B930BA40BB50B209119013091D4
:105B70001A0140911B0150911C01821B930BA40B35
:105B8000B50BBC01CD010E94892A1092320488EA2B
:105B900091E09F938F930E94BE370F900F9080915A
:105BA0003A04823009F585EE0E94EF21909133048A
:105BB000891741F088EC80933E0185EE0E94EF2129
:105BC0008093330480913E01E0911601F09117011A
:105BD000882329F4EE56FF4F80911F0104C0EE5632
:105BE000FF4F80911E01808380916A01882331F4E8
:105BF000CE0101960E94E925882361F480916A0113
:105C0000813009F0B6C2CE0101960E943726882362
:105C100009F4AFC2998190934004772069F490937E
:105C20003F0410923B0410923C0410923D041092E9
:105C30003E0470924104A0C2892F80538A3008F03C
:105C400041C080913804882371F4892F99279F934C
:105C50008F938CEA91E09F938F930E94BE370F90B1
:105C60000F900F900F9020913B0430913C04409195
:105C70003D0450913E04DA01C90163E0880F991F89
:105C8000AA1FBB1F6A95D1F7820F931FA41FB51FD0
:105C9000820F931FA41FB51F209140043327205368
:105CA0003040442737FD4095542F820F931FA41F87
:105CB000B51F80933B0490933C04A0933D04B093A4
:105CC0003E0457C29D32A9F480913804882341F4E0
:105CD0008FEA91E09F938F930E94BE370F900F90B1
:105CE00090E080914104882309F491E0909341046D
:105CF00040C29D3009F03DC2809141048823B9F033
:105D000080913B0490913C04A0913D04B0913E04ED
:105D1000B095A095909581959F4FAF4FBF4F8093C1
:105D20003B0490933C04A0933D04B0933E048091C7
:105D30003804882341F481EB91E09F938F930E9474
:105D4000BE370F900F90772480913F04863519F568
:105D500080913B0490913C04A0913D04B0913E049D
:105D6000803070E2970770E0A70770E0B7071CF07B
:105D70008FEF9FE10BC0B7FF05C010922701109273
:105D80002601F3C180913B0490913C04909327013C
:105D900080932601EAC1813421F580913B049091E2
:105DA0003C04A0913D04B0913E048030E0E29E07A7
:105DB000E0E0AE07E0E0BE071CF08FEF9FE10CC013
:105DC000181619061A061B061CF081E090E004C0A4
:105DD00080913B0490913C04909325018093240191
:105DE000C4C1823421F580913B0490913C04A09180
:105DF0003D04B0913E048030F0E29F07F0E0AF0731
:105E0000F0E0BF071CF08FEF9FE10CC018161906D9
:105E10001A061B061CF081E090E004C080913B0450
:105E200090913C0490932301809322019EC186347B
:105E3000E9F480913B0490913C04A0913D04B09121
:105E40003E0480319105A105B10514F08FE007C033
:105E5000B7FF03C07092200104C080913B0480937F
:105E60002001809120010E9497237FC18934D1F4C1
:105E700080913B0490913C04A0913D04B0913E047C
:105E80008F3F9105A105B10519F014F08FEF07C000
:105E9000B7FF03C070921F013CC080913B04809308
:105EA0001F0137C08A34D1F480913B0490913C04A7
:105EB000A0913D04B0913E048F3F9105A105B1052D
:105EC00019F014F08FEF07C0B7FF03C070921E01E6
:105ED00020C080913B0480931E011BC08B3411F5C0
:105EE00080913B0490913C04A0913D04B0913E040C
:105EF0008F3F9105A105B10519F014F08FEF07C090
:105F0000B7FF03C070921D0104C080913B048093D1
:105F10001D0140911D0160911E0180911F010E9491
:105F20009E2323C1833551F580913B0490913C041D
:105F3000A0913D04B0913E04803020E0920720E023
:105F4000A20721E0B2072CF08FEF9FEFAFEFB0E098
:105F50000CC0803040E0940740E8A4074FEFB4073E
:105F600024F480E090E0A0E8BFEF809319019093C3
:105F70001A01A0931B01B0931C01F7C0803599F55D
:105F800080913B0490913C04A0913D04B0913E046B
:105F9000803050E0950750E0A50751E0B5072CF0A0
:105FA0008FEF9FEFAFEFB0E009C080509040A04866
:105FB000BF4F64F480E090E0A0E8BFEF80933B0423
:105FC00090933C04A0933D04B0933E0480913B0425
:105FD00090913C04A0913D04B0913E04BC01CD01E0
:105FE0000E94892AC2C08D34D9F480913B049091DB
:105FF0003C04A0913D04B0913E0483309105A1057D
:10600000B10514F082E007C0B7FF03C01092390455
:1060100004C080913B04809339040E949F2AA5C04C
:10602000893561F480913B0480933804E82FFF2781
:10603000E551FF4F84918093590497C08A35D9F474
:1060400080913B0490913C04A0913D04B0913E04AA
:106050008F3F9105A105B10519F014F08FEF08C02D
:106060008197A105B10514F481E202C080913B043F
:10607000809318017AC0853551F580913B04909149
:106080003C04A0913D04B0913E0484309105A105EB
:10609000B10514F083E007C0B7FF03C010923704C6
:1060A00004C080913B048093370480913704E82F2B
:1060B000FF27E951FF4F949140E080913A048230EC
:1060C00009F441E02091360460E0892F14C0833444
:1060D00029F590913B0490933A0480913704E82F7E
:1060E000FF27E951FF4F849140E0923009F441E0ED
:1060F0002091360460E00E94CF1E80913A04E09126
:106100001601F0911701823029F4EC56FF4F84E01C
:1061100080832BC0EC56FF4F108227C0813529F5B4
:1061200080913B0490913C04A0913D04B0913E04C9
:106130000097A105B10521F081E08093360402C0EB
:106140001092360480913704E82FFF27E951FF4F62
:10615000949140E080913A04823009F441E020912A
:10616000360460E0892F0E94CF1E8EE380933F04A7
:1061700003C0772009F0AACB90913F04903209F434
:10618000A5CB209138042230C0F0809135048230B4
:10619000A0F4813041F480911801981721F482E035
:1061A0008093350402C0109235049D3011F09A306E
:1061B00051F481E08093350406C09D3011F09A308F
:1061C00021F41092350480E2FDC59E3311F09E3219
:1061D00089F42223C1F7892F99279F938F9383EB0B
:1061E00091E09F938F930E94BE370F900F900F9076
:1061F0000F90E9CF9635E1F09134D1F09634C1F0AB
:106200009934B1F09A34A1F09B3491F0933581F038
:106210009D3471F0923461F0903551F0993541F030
:10622000953531F09A3521F0933411F0913599F488
:10623000222371F4892F99279F938F9386EB91E006
:106240009F938F930E94BE370F900F900F900F90E7
:1062500001E0702E3BCB9534F9F48091B104863087
:1062600049F489EB91E09F938F930E94BE3710927F
:10627000B10409C085EC91E09F938F930E94BE37D3
:1062800086E08093B1040F900F906091B10480E09C
:1062900091E00E94DE211AC1973509F08BC08091F0
:1062A0002601909127019F938F9380ED91E09F931A
:1062B0008F930E94BE376091260181E091E00E9499
:1062C000DE216091270182E091E00E94DE21609151
:1062D000240183E091E00E94DE216091250184E0A9
:1062E00091E00E94DE216091220185E091E00E9410
:1062F000DE216091230186E091E00E94DE21609121
:10630000200187E091E00E94DE2160911F0188E07A
:1063100091E00E94DE2160911E0189E091E00E94DF
:10632000DE2160911D018AE091E00E94DE216091F2
:1063300021018BE091E00E94DE21609119018CE047
:1063400091E00E94DE2160911A018DE091E00E94AF
:10635000DE2160911B018EE091E00E94DE216091C0
:106360001C018FE091E00E94DE216091390480E100
:1063700091E00E94DE216091380481E191E00E9469
:10638000DE216091370482E191E00E94DE2160917C
:10639000180183E191E00E94DE2160913A0484E1DA
:1063A00091E00E94DE216091360485E191E00E9437
:1063B000DE21DEC2943439F0983429F09E3419F08D
:1063C0009F3409F085C00E94112B60E070E082E8E4
:1063D0009FE00E940622E0911601F0911701E05C17
:1063E000FF4F10820E947C2490932D0480932C04F4
:1063F00080912101282F332727FD30958091260198
:1064000090912701289FD001299FB00D389FB00D92
:106410001124B0933104A093300480913F04883458
:1064200021F4109231041092300480913004909144
:1064300031049F938F9380912C0490912D049F930E
:106440008F938AED91E09F938F930E94BE372091A6
:1064500030043091310480912C0490912D04EDB7DB
:10646000FEB736960FB6F894FEBF0FBEEDBF409153
:10647000240150912501281739074CF488279927C2
:10648000841B950B90932F0480932E0404C050938B
:106490002F0440932E0420E080913F048E3421F499
:1064A00021E02093450406C08F3421F422E081E0EE
:1064B0008093450440E850E06091300470913104CD
:1064C00080912E0490912F040E94A82A8EE37AC412
:1064D000973461F40E94112B60E070E080E090E05E
:1064E0000E94892A81E080933204F0CF923509F02E
:1064F000D0C00E94112BE0911601F0911701E05CD1
:10650000FF4F10820E947C24892B09F0DFC90E9472
:10651000E0237B018C016093240470932504809315
:1065200026049093270480912101992787FD909557
:10653000A92FB92F2091190130911A0140911B0107
:1065400050911C01BC01CD010E94203EDC01CB0119
:106550008E0D9F1DA01FB11F8093280490932904C6
:10656000A0932A04B0932B04BF93AF939F938F9370
:106570008091240490912504A0912604B0912704D1
:10658000BF93AF939F938F9384EE91E09F938F93EC
:106590000E94BE378091190190911A01A0911B01B0
:1065A000B0911C019C01AD01B7FF07C02227332722
:1065B000A901281B390B4A0B5B0B6DB77EB7665FD1
:1065C0007F4F0FB6F8947EBF0FBE6DBF22303105EE
:1065D000410551050CF454C04096A11DB11D819791
:1065E000A105B10508F04CC060912101862F9927C3
:1065F00087FD9095A92FB92F20912404309125046F
:106600004091260450912704280F391F4A1F5B1F11
:10661000E62FFF27E7FDF095809126019091270155
:10662000E89FB001E99F700DF89F700D11248091D3
:10663000240190912501E89FD001E99FB00DF89FBA
:10664000B00D1124CD01A0912201B091230110E8D9
:10665000E12EF12C89019A01AB01BC01EA9FC00136
:10666000EB9F900DFA9F900D11240E94D7228091EC
:10667000280490912904A0912A04B0912B04B1C060
:10668000209128043091290440912A0450912B0430
:10669000B6C0943509F0E5C00E94112BE0911601B7
:1066A000F0911701E05CFF4F10820E947C24892B3F
:1066B00009F00CC98091190190911A01A0911B0158
:1066C000B0911C01BF93AF939F938F9380EF91E0A4
:1066D0009F938F930E94BE370E94E023DC01CB0181
:1066E0002091190130911A0140911B0150911C0118
:1066F000281B390B4A0B5B0B57FF07C05095409581
:10670000309521953F4F4F4F5F4FEDB7FEB736960F
:106710000FB6F894FEBF0FBEEDBF22303105410524
:1067200051050CF464C00E94E023DC01CB012091F0
:10673000190130911A0140911B0150911C01281B35
:10674000390B4A0B5B0B57FF07C0509540953095AE
:1067500021953F4F4F4F5F4F213131054105510585
:106760000CF045C080912101282F332727FD30955B
:10677000432F532FE82FFF27E7FDF0958091260147
:1067800090912701E89FB001E99F700DF89F700D6F
:1067900011248091240190912501E89FD001E99F67
:1067A000B00DF89FB00D1124CD01A0912201B09140
:1067B000230100E8E02EF12C89019A01AB01BC0114
:1067C000EA9FC001EB9F900DFA9F900D11240E944B
:1067D000D7228091190190911A01A0911B01B091CB
:1067E0001C01AC01BD018EE00E9473226FCE20918E
:1067F000190130911A0140911B0150911C018091A7
:106800002101E82FFF27E7FDF09580912601909167
:106810002701E89FB001E99F700DF89F700D1124CA
:106820008091240190912501E89FD001E99FB00D4E
:10683000F89FB00D1124CD01A0912201B091230148
:1068400010E8E12EF12C89019A01AB01BC01EA9F0D
:10685000C001EB9F900DFA9F900D11240E94D7224A
:1068600035CE983579F488EF91E09F938F930E940D
:10687000BE3760E870E080E090E00E9496221092BF
:10688000320498C29B3241F484E092E09F938F934C
:106890000E94BE3781E009C09D3251F487E092E04A
:1068A0009F938F930E94BE378FEF8093210182C206
:1068B0009436F9F48091690490916A049F938F93C0
:1068C00080916B0490916C049F938F938AE092E087
:1068D0009F938F930E94BE378EE380933F04EDB762
:1068E000FEB736960FB6F894FEBF0FBEEDBF0C9400
:1068F000662C963649F484E00E94EF2199279F93F5
:106900008F938EE192E030C0963771F4E0911601DA
:10691000F0911701E05CFF4F10820E947C249F934E
:106920008F938DE292E020C0903791F4E0911601B0
:10693000F0911701E05CFF4F10820E94E023DC0120
:10694000CB01BF93AF939F938F9384E392E0D7C023
:106950009337B9F486E00E94EF21869586959927B2
:106960009F938F938CE392E09F938F930E94BE3707
:106970008EE380933F040F900F900F900F900C9434
:10698000662C923759F510E0E0911601F09117014D
:10699000E052FF4F108381EE0E94EF2199279F93D1
:1069A0008F9383E492E09F938F930E94BE370F9062
:1069B0000F900F900F90112359F0812F8F7041F499
:1069C00087E492E09F938F930E94BE370F900F90C1
:1069D0001F5F1034C8F289E492E0E8C1943709F0EF
:1069E000A0C08BE492E09F938F930E94BE37AA24AD
:1069F000BB2465010F900F900894A11CB11CC11C11
:106A0000D11CA89521E7E22E24E0F22E1FE30E947C
:106A10004E37DC01CB01F70181937F01115017FF45
:106A2000F6CF10E0A1E7B4E0E0911601F091170174
:106A3000E052FF4F1083E0911601F0911701EF51E2
:106A4000FF4F8D9180831F5F103470F310E091E74A
:106A5000892E94E0992EEE24FF24E0911601F09106
:106A60001701E052FF4F108381EE0E94EF21D40105
:106A70009D914D018917D9F0892F99279F938F9365
:106A800081EE0E94EF2199279F938F93FF92EF92BF
:106A900081E892E09F938F930E94BE37EDB7FEB7D7
:106AA00038960FB6F894FEBF0FBEEDBF06C01F5F4D
:106AB0000894E11CF11C103480F21034D0F0809165
:106AC0006A01882331F4CE0101960E94E9258823CA
:106AD00061F480916A01813009F08ECFCE01019678
:106AE0000E943726882309F487CF8981803209F0F4
:106AF00083CFDF92CF92BF92AF928DEA92E09F93C5
:106B00008F930E94BE378EE380933F044DB75EB7EC
:106B10004A5F5F4F0FB6F8945EBF0FBE4DBF0C9437
:106B2000662C9F3309F04DC186ED92E09F938F93C1
:106B30000E94BE370F900F908091260190912701FF
:106B40009F938F930FEF1FE11F930F931F921F923D
:106B50008AED92E09F938F930E94BE376DB77EB708
:106B6000685F7F4F0FB6F8947EBF0FBE6DBF8091F8
:106B70002401909125019F938F931F930F9381E0A0
:106B8000E82EF12CFF92EF9288EF92E09F938F9383
:106B90000E94BE378DB79EB708960FB6F8949EBF79
:106BA0000FBE8DBF80912201909123019F938F93FF
:106BB0001F930F93FF92EF9286E193E09F938F9341
:106BC0000E94BE37ADB7BEB718960FB6F894BEBFD9
:106BD0000FBEADBF8091200199279F938F9384E3CF
:106BE00093E09F938F930E94BE370F900F900F906A
:106BF0000F9080911D0199279F938F9380911E0183
:106C000099279F938F9380911F0199279F938F932B
:106C100081E693E09F938F930E94BE37EDB7FEB756
:106C200038960FB6F894FEBF0FBEEDBF80911901E4
:106C300090911A01A0911B01B0911C01BF93AF93D9
:106C40009F938F9380EA93E09F938F930E94BE3728
:106C50004DB75EB74A5F5F4F0FB6F8945EBF0FBE89
:106C60004DBF8091390499279F938F938FEB93E0C9
:106C70009F938F930E94BE370F900F900F900F90AD
:106C80008CEE93E09F938F930E94BE370F900F90EE
:106C900087E094E09F938F930E94BE370F900F90F0
:106CA00080E294E09F938F930E94BE370F900F90E5
:106CB00081E394E09F938F930E94BE370F900F90D3
:106CC00080912101992787FD90959F938F9382E66C
:106CD00094E09F938F930E94BE370F900F900F9078
:106CE0000F908AE794E09F938F930E94BE370F9096
:106CF0000F9080913A0499279F938F9380EA94E0B4
:106D00009F938F930E94BE370F900F900F900F901C
:106D10008091380499279F938F9389EC94E09F93F7
:106D20008F930E94BE370F900F900F900F9080911D
:106D3000180199279F938F9385EF94E09F938F93EA
:106D40000E94BE370F900F900F900F9080913704E4
:106D500099279F938F9389E095E09F938F930E944B
:106D6000BE370F900F900F900F90809136049927A7
:106D70009F938F9388E395E09F938F930E94BE37F4
:106D80000F900F900F900F908AE595E09F938F934F
:106D90000E94BE370F900F9085E795E09F938F93E9
:106DA0000E94BE370F900F908BE895E09F938F93D2
:106DB0000E94BE378EE380933F040F900F900C9497
:106DC000662C8EE280933F040C94662CAF92BF92A7
:106DD000CF92DF92EF92FF920F931F93CF93DF93A7
:106DE000EC01E880F9800A811B81C801B7012DE11F
:106DF00033EF41E050E00E943F3E59016A01C80173
:106E0000B7012DE133EF41E050E00E943F3EDC014D
:106E1000CB01BC01CD0127EA31E440E050E00E9403
:106E2000203E7B018C01C601B50124E13BE040E03E
:106E300050E00E94203EDC01CB01E81AF90A0A0B5F
:106E40001B0B1E141F041006110644F08FEF9FEF5A
:106E5000AFEFBFE7E80EF91E0A1F1B1FE882F98299
:106E60000A831B838FEF9FEFAFEFBFE7E822F92282
:106E70000A231B23C801B701DF91CF911F910F9106
:106E8000FF90EF90DF90CF90BF90AF9008950E9459
:106E9000E636DC01CB01BC01CD01089582E391E02F
:106EA0000E94E636DC01CB01BC01CD010895DC0176
:106EB000CB018093320190933301A0933401B093BE
:106EC000350108950F931F93CF93DF938C01EB014E
:106ED000009711F4672BC1F16EE070E081E090E063
:106EE0000E94A03AFC01892B71F180E883832097EE
:106EF00071F0D387C28781E883838091B204909137
:106F0000B304892B21F4F093B304E093B204011588
:106F10001105C9F011870087838182608383809186
:106F2000B4049091B504892B71F4F093B504E09307
:106F3000B4048091B6049091B704892B21F4F093A6
:106F4000B704E093B604CF01DF91CF911F910F9169
:106F50000895CF93DF93CDB7DEB7E5E0F0E0EC0F17
:106F6000FD1F81919191AF01BC018091B40490917A
:106F7000B5040E94E337DF91CF910895CF93DF935B
:106F8000CDB7DEB745E050E04C0F5D1FFA0121910F
:106F90003191AF01A091B404B091B504FD0183819A
:106FA00088608383B9018091B4049091B5040E94F4
:106FB000E337E091B404F091B5042381277F238364
:106FC000DF91CF9108952F923F924F925F926F92EF
:106FD0007F928F929F92AF92BF92CF92DF92EF9269
:106FE000FF920F931F93CF93DF93CDB7DEB76297D6
:106FF0000FB6F894DEBF0FBECDBFEE24FF2487018D
:107000001C017E876D872A01CC24DD24FC01D782F8
:10701000C682838181FD68C28FEF9FEF78C28D8524
:107020009E8501969E878D87C0FE4BC28F858053BB
:107030008A30D0F49F85903339F4662029F4C3FC5C
:1070400003C0E0E0F1E08DC08AE0689E602C11246E
:10705000FF856F0E20ED620E67FE02C05FE7652EB2
:10706000C3FC42C2762C40C2C3FE04C0662011F4A9
:1070700041E0642EEF858E2F992787FD9095883605
:1070800091058CF5853691050CF06EC08335910520
:1070900009F493C084359105CCF48B32910509F441
:1070A00049C08C3291054CF48032910509F446C0F8
:1070B0008332910509F44AC0FEC18D32910509F46D
:1070C00040C08E32910509F444C0F5C18336910564
:1070D00009F450C0843691050CF08AC088359105BA
:1070E00009F4BCC0E8C18037910509F4B1C081370B
:1070F000910584F48C36910591F18D3691052CF42F
:107100008936910509F474C0D6C18F36910509F40A
:107110009CC0D1C18537910509F4A2C0863791057D
:1071200024F48337910571F1C6C18837910509F4BC
:1071300095C0C1C180E190E0C82AD92AE0E2F0E020
:1071400010C080E890E0C82AD92ACEC1E0E4F0E07F
:1071500008C088E090E0C82AD92A6624C5C1E4E0C6
:10716000F0E0CE2ADF2AC0C13FE3E32E7A94F3E6B3
:10717000FF873CC1F20182E090E0480E591EE0809A
:107180007A9434C1F20182E090E0480E591EA08149
:10719000B1817D01C3FE09C0862D992787FD909599
:1071A000BC01CD010E94D03B1FC0FD010190002019
:1071B000E9F73197EA1BE88B18C0F20182E090E012
:1071C000480E591E0190F081E02D7F01C3FE09C0D9
:1071D000862D992787FD9095BC01CF010E94BB3B6E
:1071E00003C0CF010E94B23B888B9889791AFEC0F8
:1071F000C2FE0AC0F20184E090E0480E591E2081D0
:107200003181428153810CC0F20182E090E0480E4E
:10721000591E808191819C01442737FD4095542F50
:1072200079018A0157FF0CC0E2E0F0E0CE2ADF2AA4
:1072300010950095F094E094E11CF11C011D111DC6
:107240008FEB9FEFC822D92227C098E0988B08C007
:10725000E0E4F0E0CE2ADF2AF8E7FF8720E1288B80
:10726000C2FE0AC0F20184E090E0480E591E20815F
:107270003181428153810AC0F20182E090E0480EE0
:10728000591E808191819C014427552779018A01EB
:10729000EFECFFEFCE22DF22CE0101969A8B898B95
:1072A0009889892E9924AA24BB24C801B701A50175
:1072B00094010E943F3EDC01CB01E989FA89808379
:1072C0008A3024F0FF858F0F815201C0805DE989EB
:1072D000FA898193FA8BE98BC801B701A501940162
:1072E0000E943F3E79018A01211531054105510572
:1072F000E1F6E98881E090E08C0F9D1FE81AC60155
:1073000082739070892B09F07A94C6FE0DC0872D88
:10731000992787FD9095E889E03121F42EEF722EB0
:10732000780E02C0782E7A94C3FE0FC0262D332724
:1073300027FD30958E2D9927821793072CF087EF24
:107340009FEFC822D92201C06E18C3FE02C0761872
:1073500001C07E18C60180789170892B51F4872D69
:107360007A94181634F4B10180E290E00E94DB3B7D
:10737000F6CFC1FE04C0B1018DE290E00BC0C4FEA7
:1073800004C0B1018BE290E005C0C5FE05C0B101AB
:1073900080E290E00E94DB3BC6FE10C0B10180E3BA
:1073A00090E00E94DB3B9889903141F4B101EF8578
:1073B0008E2F992787FD90950E94DB3BD0FE0AC057
:1073C000872D7A94181634F4B10180E390E00E947E
:1073D000DB3BF6CFC3FE0AC0862D6A94181634F440
:1073E000B10180E390E00E94DB3BF6CF90E8B92E3C
:1073F000BC2051F4872D7A94181634F4B10180E240
:1074000090E00E94DB3BF6CFFF85F33641F48E2DF2
:10741000B101992787FD90950E94DB3B40C02F85E5
:107420002337B1F488898150888B8F3FC1F1F701F0
:1074300080810894E11CF11CB101992787FD90958A
:107440000E94DB3B98899150988B9F3F81F727C022
:10745000EF85E33579F4F889F150F88BFF3FF9F0C7
:10746000F7018491B10199270E94DB3B0894E11C4C
:10747000F11CF1CF6E010894C11CD11C89899A8935
:107480008C159D0561F0E989FA898291FA8BE98B67
:10749000B101992787FD90950E94DB3BEFCFBB2080
:1074A00069F0872D7A9418164CF4B10180E290E0CF
:1074B0000E94DB3BF6CFB1010E94DB3BCC24DD24F4
:1074C00013C09F85953241F481E0C82ED12C6624EB
:1074D000762CEAE0E88B08C0B101FF858F2F992751
:1074E00087FD90950E94DB3BF101838183FF04C0FF
:1074F000ED85FE85F49103C0ED85FE85F081FF8763
:107500002F85222309F08BCDF10186819781629628
:107510000FB6F894DEBF0FBECDBFDF91CF911F91A4
:107520000F91FF90EF90DF90CF90BF90AF909F9022
:107530008F907F906F905F904F903F902F90089525
:107540000F931F93CF93DF93869F8001879F100D2A
:10755000969F100D1124C8010E94BC3AEC010097BF
:1075600029F0A80160E070E00E94C63BCE01DF91E7
:10757000CF911F910F910895CF93DF93AC010297A4
:1075800010F442E050E020E030E0A091BA04B09165
:10759000BB04BD01F901109709F44CC08D919C9179
:1075A00011978417950731F14817590738F42115B9
:1075B000310519F08217930708F49C01FD01A2819F
:1075C000B381109759F721153105A1F1C901841B29
:1075D000950B049708F4A901DB01E0E0F0E01097B7
:1075E00049F18D919C91119782179307F9F44217F5
:1075F000530779F4ED018A819B81309719F09383C9
:10760000828304C09093BB048093BA04CD01029698
:107610004AC0241B350BFD01E20FF31F4193519328
:10762000225030402D933C93CF013DC0FD01A281FB
:10763000B381D5CF8091B8049091B904892B41F4DE
:1076400080913801909139019093B9048093B804E6
:10765000E0913601F0913701309741F4EDB7FEB774
:1076600080913A0190913B01E81BF90BA091B8047D
:10767000B091B9049F012A1B3B0B2417350788F0F2
:10768000CA0102962817390760F0CD01840F951FB3
:1076900002969093B9048093B8044D935D93CD0105
:1076A00002C080E090E0DF91CF910895CF93DF9307
:1076B000009709F454C0DC011297ED011B821A8275
:1076C0008091BA049091BB04009721F1FC0140E045
:1076D00050E0EA17FB0718F1ED01FB83EA832D91D7
:1076E0003C911197C20FD31FCE0102968E179F07B0
:1076F00071F48A819B81280F391F2E5F3F4F1196AD
:107700003C932E9382819381FD0193838283411563
:10771000510559F4B093BB04A093BA0420C0AF0143
:107720000280F381E02D3097A1F6EA01BB83AA83A2
:10773000CA01029628813981820F931F8A179B07FD
:1077400071F48D919C911197280F391F2E5F3F4F37
:1077500039832883FD01828193819B838A83DF9112
:10776000CF910895FC0105900020E9F78095909550
:107770008E0F9F1F0895FC0105906150704001100D
:10778000D8F7809590958E0F9F1F0895DC0140FFDC
:1077900003C001C06D936D9342505040D8F70895D7
:1077A000FC016150704001900110D8F780959095D0
:1077B0008E0F9F1F08950F931F93CF93DF938C011C
:1077C000EB018B81992781FF1CC082FF0DC02E81A8
:1077D0003F818C819D812817390764F4E881F98104
:1077E0000193F983E88306C0E885F985802F099520
:1077F000892B39F48E819F8101969F838E83C801E6
:1078000002C08FEF9FEFDF91CF911F910F910895ED
:107810005058192EEFD001D0D2C0BA1762077307A3
:1078200084079507B1F188F40EF410940B2EBA2F4B
:10783000A02D062E622F202D072E732F302D082EFF
:10784000842F402D092E952F502DFF275523B9F059
:10785000591B49F0573E98F0469537952795A795BF
:10786000F0405395C9F776F0BA0F621F731F841F5B
:1078700030F4879577956795B795F040939517FA0B
:107880000F2E0895BF1BBB27BA0B620B730B840B23
:10789000F6CFDEF6DBC0AED001D091C0552359F053
:1078A000992369F09F575F57951B33F442F4903842
:1078B00011F4915805C09BC091589F3F09F4C6C070
:1078C000BB27112462177307840730F4660F771FF4
:1078D000881FBB1F915098F311D00F920FD00F92B9
:1078E0000DD0A0E82617370748071B0609F0A04867
:1078F000BA2F602D7F918F9100240895A0E8002475
:10790000621773078407B10528F0621B730B840BA1
:10791000B1090A2A660F771F881FBB1FA69581F73A
:10792000089597FB73D09F3738F0FEE9F91B982F25
:10793000872F762F6B2F05C086C0969587957795F4
:107940006795F150D0F73EF49095809570956195CC
:107950007F4F8F4F9F4F0895E89403C097FB0EF41D
:10796000F3DFB62F672F782F892F9EE9002427C0D9
:107970000ED05EF004C00BD026F001C008D019F084
:1079800020F48FEF089580E0089581E0089597FB3B
:10799000092E052600F8689430D0E89407FC07C04B
:1079A000621773078407950721F008F40094079481
:1079B000989408959A95BB0F661F771F881F11240E
:1079C0009923A1F08823B2F79F3F59F0BB0F48F4E9
:1079D00021F4002011F460FF04C06F5F7F4F8F4FD0
:1079E0009F4F881F9795879597F908952CC09FEF13
:1079F00080EC0895052E092607FA440F551F5F3FB6
:107A000079F0AA27A51708F051E04795880F991F2C
:107A10009F3F31F0BB27B91708F091E08795089593
:107A20009F919F911124E3CF97FB880F991F9F3F50
:107A300031F0BB27B91708F091E0879508959F9121
:107A40009F911124D4CF66277727882799270895F7
:107A5000D1DF01D0B4CF992339F0552329F09F57B6
:107A60005F57950F13F49AF1F1CF91589F3FE1F3CF
:107A7000629FA12D0F92BB27639FA00DB11DEE2722
:107A8000729FA00DB11DEE1FAF93AA27649FB00D8A
:107A9000E11D739FB00DE11DAA1F6627829FB00DE7
:107AA000E11DA61F5527749FE00DA11D551F839F43
:107AB000E00DA11D561F849FA00D511D852F7A2F0B
:107AC0006E2F1F900F9088231AF4939539F48FCF5F
:107AD000000C111CBB1F661F771F881F012808950B
:107AE0009F939F77993358F050E449EC3FE02BED9A
:107AF0000AD05FEB49EC3FE02BED8BDE17D05F91B6
:107B00005078952708955F77552319F444230AF098
:107B10006ECF2F933F934F935F93BDDE552744273E
:107B200056D05F914F913F912F9192CF1F939F77A6
:107B300050EC49E43FE02BED6CDE10E89F775FE30B
:107B400049EC3FE02BED621773078407950720F09F
:107B500050EC49E45EDE11276AD09068E4E9F0E079
:107B600003D091271F910895FF92EF92DF92CF9259
:107B7000BF926B017C01B59016D0B590BB2069F027
:107B80009F938F937F936F93B601C7010CD02F9172
:107B90003F914F915F910E944B3CBF90CF90DF90FF
:107BA000EF90FF90089547D002C09601A701EF9390
:107BB000FF930E94283DFF91EF913DD0EF93FF93FB
:107BC0000E94093CFF91EF91BA9479F708952CDF58
:107BD000CF93DF93D52FC42F552744273327222750
:107BE0009923D9F09F37C8F0F92FE9DE592F482F94
:107BF000372F262FF63968F494DEB0DEC030CD077B
:107C000021F069937993899399939058DF91CF915B
:107C100000CE9927882777276627C030CD0721F027
:107C20002993399349935993DF91CF91C8CE9B0102
:107C3000AC010C94283D55914591359125910895BD
:107C4000629FD001739FF001829FE00DF11D649F40
:107C5000E00DF11D929FF00D839FF00D749FF00DCC
:107C6000659FF00D9927729FB00DE11DF91F639F6D
:107C7000B00DE11DF91FBD01CF0111240895A1E24E
:107C80001A2EAA1BBB1BFD010DC0AA1FBB1FEE1F96
:107C9000FF1FA217B307E407F50720F0A21BB30BE1
:107CA000E40BF50B661F771F881F991F1A9469F75D
:107CB00060957095809590959B01AC01BD01CF01B9
:107CC000089597FB092E05260ED057FD04D0D7DF67
:107CD0000AD0001C38F450954095309521953F4FBF
:107CE0004F4F5F4F0895F6F7909580957095619589
:087CF0007F4F8F4F9F4F089555
:107CF80001006401410100000064000101E80388FB
:107D08001364000A000100114188130000FFC864D1
:107D180007010A006400FF1F256420746F20256492
:0C7D28000A00010000000000BC04200064
:00000001FF
